:100000000C9443040C946B040C946B040C946B04DC
:100010000C946B040C946B040C946B040C946B04A4
:100020000C946B040C947A050C9410280C94FB36F9
:100030000C946B040C9477340C94B5340C946B04CE
:100040000C9478060C946B040C946B040C946B0465
:100050000C946B040000000048A50C4C000000004C
:100060007C6B0831850032007D09E8038000320096
:1000700057012C0100000000C0AE4E5AFC53501432
:100080003FA0540B00000000A8D5803E80186009F6
:10009000DC377017000000000000000000000000C6
:1000A00040C7370F0000000080C7300F000000007D
:1000B00040CA310F00000000E1C7340F000000000B
:1000C000B7C6400F00000000B7C6400F0300320063
:1000D0005600E803090032001A002C01FF0000005E
:1000E0000005040000040900FF01010001050500EE
:1000F00001040A00FF0202000205060002040B00D0
:10010000FF0000000305070003040C00FF030300C9
:100110000405110204040D00FF020200050511048C
:1001200005040E0006051101070511088D0C880C49
:10013000D30D2020436865616C694368617267650F
:100140007200202020207665723A20302E33320053
:10015000540100006F7074696F6E7300010001003C
:100160000100010001000A00640001000200040017
:100170001000400000010004010003000800070017
:10018000070014000700496E660079657300206E51
:100190006F006D560047024F02540259025D026221
:1001A0000267026C0201000100010001000000B0C2
:1001B000041C07520300000807B0044006E80300CF
:1001C000000807D0079209D60600000000E40C10D2
:1001D0000ED007E40C0000100E0410C409A60E0097
:1001E00000740E6810B80B0A0F000040066C07146C
:1001F000054006000000980898086C071027019831
:100200000898086C07010002980898086C0701001C
:10021000039808DC006C07060004980898086C072F
:10022000030005980898086C0703000698089808CA
:100230006C07030007980898086C070300756E6C3C
:10024000696D6974656400556E6B6E6F776E004EF4
:10025000694364004E694D480050623F004C696636
:1002600065004C696C6F004C69706F004E695A6E86
:1002700000920299029E02A302A802AD02BB0200F4
:100280000045646974206E616D653A004E616D656C
:100290003A004261743A202000563A202000436818
:1002A0003A200049633A200049643A200020206344
:1002B0007265617465206E616D6500202020656443
:1002C0006974206E616D650043684342426C446905
:1002D00046435374534243684469437943594368DE
:1002E000446945420020202D2D2020004C696D6975
:1002F00074733A200074696D653A20202020200034
:10030000622000202000626174742E20523D00772C
:100310006972657320523D0056696E7075743D00B8
:10032000206C696D69743D00566F7574203D0056F0
:1003300062616C2E3D00546578743D002D00546957
:100340006E743D0070726F6772616D20636F6D70C7
:100350006C65746500726561736F6E3A20006D6F35
:100360006E69746F72206572726F72006E6F7420A6
:1003700075736564006D6178566F75743D006465D2
:100380006C746120563D2000546578743D006E6F9A
:100390007420757365640064656C746120543D203D
:1003A0000046756E6374696F6E206E6F7400696DC0
:1003B000706C656D656E7465642079657400706C31
:1003C000656173652063616C696272617465006266
:1003D00065666F72652075736500524556455253C8
:1003E0004520504F4C41524954590046554C20002D
:1003F000252000901F841F941F56206C696D69741E
:10040000002D64560064542F647400592062202526
:10041000208A209120D020352103210921E421F2D6
:10042000216621010607050002060708090B0C0DCD
:100430000405030002060708090B0C0D0405030060
:10044000020A0E0F0B0C0D04050300020607080933
:100450000B0C0D04050300020F0B0C0D040503002B
:1004600006070405000000010203040D0001020359
:100470000405060D0708090A0D0B0C0DB004B7049E
:10048000C604CE04D804E404EC04FB040000B00469
:10049000CE0408051205FB040000B004B704C6042E
:1004A000CE04D804FB040000B004CE04FB0400001A
:1004B000636861726765006368617267652B62617A
:1004C0006C616E63650062616C616E636500646996
:1004D0007363686172676500666173742063686145
:1004E0007267650073746F726167650073746F7211
:1004F0006167652B62616C616E630065646974207D
:100500006261747465727900633E64206379636C20
:100510006500643E63206379636C6500696E746591
:10052000726E205400626174206469736300696EA6
:1005300070757420560063617020434F4646006515
:1005400078742054434F4600436F6E6E6563742089
:10055000426174746572792100B305B905BF05C5A0
:1005600005CB05D105D705DD05E3050000061E1FF7
:1005700020212223120006090A0B0C0D0E76616C55
:1005800075653A2000496F75743A202000E905EE40
:10059000050000E905F5050000FB0502060000095D
:1005A00006120600001B0623062C063806440650D9
:1005B00006000056696E3A20005662313A20005615
:1005C00062323A20005662333A20005662343A20B2
:1005D000005662353A20005662363A200056312DD8
:1005E000363A00566F75743A0035306D410031303F
:1005F00030306D41003330306D410074656D703ABC
:10060000200076616C75653A00706F696E742031F8
:100610002E00706F696E7420322E00766F6C7461DC
:1006200067650049206368617267650049206469F5
:10063000736368617267650074656D7020657874B6
:1006400065726E0074656D7020696E7465726E00FF
:1006500063616C69622D3E554152540064066D061B
:100660007706000073657474696E67730063616C6C
:100670006962726174650072657365742064656691
:1006800061756C740080250000004B00000096002E
:100690000000E1000000C20100460088137017014D
:1006A000007017640007000C0005007800581B005C
:1006B00000080000000300E706F206FD0608071424
:1006C000071F07260730073A07460750075B0764EE
:1006D000076E0775077D070000432F6D0086078FA3
:1006E0000796079C07A5076261636B6C696768746E
:1006F0003A0066616E206F6E3A20202000646973B4
:100700006368206F66663A00657874726E20543AAA
:1007100020202000657874726E2054434F3A0064A4
:10072000542F64743A004E694D48202D64563A00A7
:100730004E694364202D64563A00432F4420637968
:10074000636C65733A0063617020434F66663A00DC
:10075000696E707574206C6F773A006469736368B2
:10076000202B3A0062616C2E206572723A0055416E
:1007700052543A200073706565643A2000202020AE
:1007800072657365740064697361626C6564006EA0
:100790006F726D616C006465627567006578742EB8
:1007A00020646562006578742E204164630013162E
:1007B0001817190705061E1F20212223726573656D
:1007C00074696E6720656570726F6D3A00763A20C5
:1007D000372E312E32200063200064200073200069
:1007E0000000000000000000000000000004030002
:1007F00005000000000000000000000000000000F4
:100800000000000000000000000001000000204087
:100810008000000000000102040810204080000059
:1008200001020408102040800000008040201008D1
:10083000040201000001020408100002020200008C
:10084000000000040404040404040400000303037F
:100850000303030303000000010101010101010181
:100860000000020202020200003B003800350032A4
:100870000000003A00370034003100006705400FE7
:10088000581F7924A73511241FBECFE5D8E0DEBF5D
:10089000CDBF10E0A0E6B0E0E0EFF1E702C00590C8
:1008A0000D92A03EB107D9F714E0A0EEB0E001C070
:1008B0001D92AC39B107E1F718E0C6E8D8E004C0F2
:1008C0002297FE010E947D38CC37D107C9F70E94DC
:1008D00063360C94F6380C940000CF92DF92EF92BE
:1008E000FF920F931F93482F282F30E0A8EBBBE017
:1008F0000E94EF376B017C01A4E6B0E0A41BB109B4
:1009000024E630E00E94FB376C0D7D1D8E1D9F1D7F
:1009100024E630E040E050E00E943D3869017A0171
:100920000FEF1FEF9801A6016DE085EF90E00E94A8
:1009300022061F910F91FF90EF90DF90CF900895C6
:10094000682F89E00C94B837BC0180E10C94B7366D
:1009500061E068278CE00C94B83761E068278FE08D
:100960000C94B83761E068278BE00C94B8370F938C
:100970001F930FEF1FEF9801AC016EE085EF90E041
:100980000E9422061F910F9108950F931F930FEF5E
:100990001FEF9801AC016EE085EF90E00E94220607
:1009A0001F910F910895CF93C82F682F617088E22F
:1009B0000E94B8376C2F627089E20E94B8376C2FA2
:1009C00064708AE20E94B8376C2F68708BE20E94D4
:1009D000B8376C2F60718FE10E94B8376C2F60724E
:1009E0008EE1CF910C94B83761E08DE00E948037A2
:1009F00061E08CE00E94803761E089E00E948037EE
:100A000061E080E10E94803761E088E20E948037E7
:100A100061E089E20E94803761E08AE20E948037CB
:100A200061E08BE20E94803761E08FE10E948037B5
:100A300061E08EE10E94803761E08EE00E948037A5
:100A400061E08FE00E94803761E08EE00E94803795
:100A500061E08BE00E94803761E083E00E94803794
:100A600061E082E00E94803761E081E00E9480378F
:100A700060E080E20E94803760E081E20E9480377F
:100A800080E00E94A80480E00E94A00480E090E042
:100A90000E94A40480E00E94D30420E042E060E1D0
:100AA00080EE90E00E948B150E94DA270E94492276
:100AB0000E94C72240E052E060E070E085EF90E0E5
:100AC0000E9402060E940F070C94DA0B0895CF9241
:100AD000EF920F9383E1C82E94E1E92E05E126E120
:100AE00047E168E180EE90E00E943F160F91EF90A1
:100AF000CF9008951F920F920FB60F9211242F934B
:100B00003F934F935F936F937F938F939F93AF9395
:100B1000BF93EF93FF93E091F800F091F9000995EE
:100B2000FF91EF91BF91AF919F918F917F916F91C5
:100B30005F914F913F912F910F900FBE0F901F909B
:100B40001895FC01A3E0440F551F661F771FAA9557
:100B5000D1F74115510581E06807710514F481E072
:100B60000EC033E075956795579547953A95D1F73F
:100B70004115510581E0680771051CF482E082830C
:100B800032C023E075956795579547952A95D1F71B
:100B90004115510581E06807710514F483E0EFCF3A
:100BA00092E075956795579547959A95D1F74115B8
:100BB000510581E06807710514F484E0E0CF82E01C
:100BC00075956795579547958A95D1F785E0828306
:100BD0004115510581E0680771050CF404C04FEF21
:100BE0005FEF60E070E08FB7F8945183408357BDAA
:100BF00046BD8FBF8EB5887F8EBD8EB59281892B05
:100C00008EBD08951FBC20E12EBD0C94A1058FB7A9
:100C1000F894613021F0693011F06E3019F45BBD49
:100C20004ABD08C0623021F06A3011F06D3011F415
:100C300059BD48BD8FBF08952EB5FC018281282B78
:100C40002EBD0895DF92EF92FF920F931F93CF93E3
:100C5000DF93EC01D62E7A01101611061206130648
:100C600024F4B901A8010E94A10581E0D81631F051
:100C700089E0D81619F08EE0D81203C08FB58068CD
:100C80000BC082E0D81631F08AE0D81619F08DE05A
:100C9000D81203C08FB580628FBDA7016D2DCE0124
:100CA0000E940706CE01DF91CF911F910F91FF9017
:100CB000EF90DF900C941C06909160008917B9F0BA
:100CC0008093600098B3282F217030E0220F331FEB
:100CD000220F331F82FB332730F9232B8270282BFE
:100CE00080E2289F900111249F71922B98BB089558
:100CF0001F920F920FB60F9211240F900FBE0F90FC
:100D00001F9018958091FA0008951092FB00EDED68
:100D1000F0E0E491E770E062E7B990E084E0989F4A
:100D2000F0011124E452FF4F8491933111F09F5F41
:100D300001C090E087FDF2CF0C945C06369A0895CE
:100D40000E940D229093C3018093C2010E945F22F2
:100D50009093C5018093C4010C94480BCF93DF930B
:100D6000D82F84B195B12091FB0044E0249F9001DD
:100D70001124F901E252FF4FE491E13171F04FB7D4
:100D8000F894F0E0EE0FFF1FEC55FE4F392F20E0F6
:100D9000282B318320834FBF0EC0F901E152FF4F52
:100DA00024913091FA0097FD02C0232B02C02095B8
:100DB00023232093FA00C091FB00C33111F0CF5FD1
:100DC00001C0C0E0C093FB009C2F84E0989FF0011D
:100DD0001124E452FF4F8491933111F09F5F01C0C1
:100DE00090E087FDF2CF0E945C0644E0C49FF001D2
:100DF0001124E352FF4FE491E770E062E7B9DD238D
:100E000041F08091FB00811104C0DF91CF910C94DF
:100E1000A0068EE190E0DF91CF910C94453761E020
:100E200083E00E94803761E082E00E94803761E0C9
:100E300081E00E9480378FE886B90C9485060E9475
:100E40009E063699FECF0E947A070C94AE060C944B
:100E50008506CF93DF930E94A5090E943B09C091AC
:100E60001201D091130102C00E941F07809112014C
:100E700090911301C817D907B9F3DF91CF91089565
:100E8000CF92DF92EF92FF92CF93DF93EC010E941B
:100E900034286B017C01CC0EDD1EE11CF11C0E948C
:100EA0001F070E9434286C157D058E059F05B8F339
:100EB000DF91CF91FF90EF90DF90CF900895E82FD2
:100EC000F0E0EE0FFF1FEA53FE4F808191810895FD
:100ED000E82FF0E0EE0FFF1FE45AFE4F8081918172
:100EE0000895E82FF0E0EE0FFF1FEC55FE4F8081D4
:100EF0009181089580912E02089580911201909120
:100F000013010895E82FF0E0EE0FFF1FEC5EFE4F97
:100F1000808191810895262F613110F4423040F094
:100F200021E030E0FC013383228331832083089564
:100F3000642F70E0F2E02F9F600D711D1124660F89
:100F4000771F660F771F6E5F7F4F44E050E00C9471
:100F5000B138282FCA01213190F4623080F470E05A
:100F600032E0239F600D711D1124660F771F660FFD
:100F7000771F6E5F7F4F44E050E00C94CF380895A8
:100F8000FF920F931F93CF93DF9300D000D0CDB784
:100F9000DEB7F12C88E0F89E80011124F801EC5AAC
:100FA000FF4F459155916591749149835A836B83A5
:100FB0007C83AE014F5F5F4F60E08F2D0E94A907D9
:100FC000F801E85AFF4F4591559165917491498315
:100FD0005A836B837C83AE014F5F5F4F61E08F2D3F
:100FE0000E94A907F39481E1F812D4CF0F900F90DB
:100FF0000F900F90DF91CF911F910F91FF90089567
:10100000E82FF0E0EE0FFF1FE45AFE4F2081318100
:10101000E82FE250E53170F4F0E0E459FF4F8081B1
:10102000882319F0813061F405C081E02333310554
:1010300040F404C081E0293E334018F480E0089574
:1010400081E00895CF93C0E08C2F825E0E9400085B
:10105000882319F0CF5FC630B9F78C2FCF91089550
:1010600020918801309189018091FC009091FD00D0
:10107000A091FE00B091FF00820F931FA11DB11D32
:101080008093FC009093FD00A093FE00B093FF00BE
:1010900008956091FC007091FD008091FE00909198
:1010A000FF002DE730E040E050E00E943D38772718
:1010B000652F542F432FCA010895E2E8F1E08081A3
:1010C0009181089580913A0190913B01039750F0EE
:1010D0008091400190914101039720F083E090E0DE
:1010E0000C94050D80E0089590E0880F991FFC0195
:1010F000E45AFE4F208131816217730718F4261BD2
:10110000370B04C0AB01421B530B9A01FC01EC5E90
:10111000FE4F2730310518F01182108206C0208161
:1011200031812F5F3F4F31832083FC01E45AFE4F12
:10113000718360830895AF92BF92CF92DF92EF9256
:10114000FF920F931F93CF93DF931F92CDB7DEB71C
:10115000A0905C01B0905D010EE611E09EE1F80107
:10116000619171918F01892F99830E9474089981EF
:101170009F5F9432A1F70E942208082F80E0E12CA3
:10118000F12C0CC0E82FE25EF0E0EE0FFF1FE45AF6
:10119000FE4F20813181E20EF31E8F5F8013F2CF6C
:1011A000B70182E10E947408E114F10449F0EA14E5
:1011B000FB0448F495012E193F09293E334018F0ED
:1011C00010E000E002C0570112E1B50183E10E9486
:1011D0007408602F70E085E10E947408612F70E050
:1011E00084E10E9474080E9449088C010E945022E8
:1011F000882329F0E0906201F09063010BC00E9407
:10120000FE21882329F0E0906001F090610102C086
:10121000E12CF12CB70186E10E947408B80188E145
:101220000E9474089701D5010E94EF3730E1C32E68
:1012300037E2D32EE12CF12CA70196010E943D3814
:10124000B90187E10E9474089801D5010E94EF3727
:10125000A70196010E943D38B90189E10F90DF9105
:10126000CF911F910F91FF90EF90DF90CF90BF90A3
:10127000AF900C94740810922D0210922C0280E012
:1012800094E0899FF0011124E851FE4F10821182F1
:10129000128213828F5F813199F7089510920F01A6
:1012A00010920E0110920A0110920B0110920C0183
:1012B00010920D0110920601109207011092080180
:1012C0001092090110921101109210011092050163
:1012D000109204010E943428609300017093010170
:1012E0008093020190930301089580E0E82FF0E0DD
:1012F000EE0FFF1FEC5EFE4F118210828F5F843273
:10130000A9F708950E943B090C94750910921301E6
:10131000109212011092FC001092FD001092FE003B
:101320001092FF000E9427070E9482090E944E0926
:1013300080E0E82FF0E0EE0FFF1FE45AFE4F11822D
:1013400010828F5F8432A9F7089580912E02811157
:101350000AC081E00E94A8040E94860981E080936F
:101360002E020C942907089510922E0280E00C940E
:10137000A8042091A6013091A7018091A401909129
:10138000A5018217930718F4281B390B02C020E02F
:1013900030E081E0293E334008F480E008958F92E8
:1013A0009F92AF92BF92CF92DF92EF92FF92CF9334
:1013B000DF93CDB7DEB728970FB6F894DEBF0FBE28
:1013C000CDBFF82E5B0140E0682FCE0105960E944C
:1013D0008B0741E06F2DCE0101960E948B072B8178
:1013E0003C8140E050E0CF80D884E12CF12C2C19D6
:1013F0003D094E095F09B50180E090E08D809E8037
:10140000A12CB12C681979098A099B090E940D3811
:1014100029813A8140E050E0281939094A095B09DD
:101420000E945F382C0D3D1D4E1D5F1D57FF03C0F0
:1014300020E030E0A901C90128960FB6F894DEBF7C
:101440000FBECDBFDF91CF91FF90EF90DF90CF9097
:10145000BF90AF909F908F9008951F93CF93DF938D
:101460008091120190911301019690931301809342
:10147000120110E0C12FD0E0DE01AA0FBB1FAA0F9E
:10148000BB1FA851BE4F20912C0230912D0240E08D
:1014900050E06D917D918D919C910E943D38FE01AF
:1014A000EE0FFF1FEA53FE4F31832083B901812FD6
:1014B0000E94CF09BC01812F0E9474081F5F113167
:1014C000C9F60E949B080E943A33DF91CF911F9189
:1014D0000C943B090F931F93CF93DF93C1E02091AE
:1014E00084013091850180910A0190910B01A091B6
:1014F0000C01B0910D012231310531F0C0E0209195
:10150000A4013091A50104C0209182013091830192
:10151000820F931FA11DB11D80930A0190930B01AF
:10152000A0930C01B0930D012091B2013091B30151
:101530008091060190910701A0910801B0910901E5
:10154000820F931FA11DB11D809306019093070187
:10155000A0930801B093090180910E0190910F01B1
:10156000019690930F0180930E010E943428009100
:101570000001109101012091020130910301601BD3
:10158000710B820B930B61367A4E8105910508F43D
:101590007AC08091100190911101019690931101F0
:1015A0008093100120910E0130910F0140E050E036
:1015B00060910A0170910B0180910C0190910D01D5
:1015C0000E943D3810920A0110920B0110920C01FA
:1015D00010920D01C11106C0B90180E00E94CF092F
:1015E0008C0101C08901C0919201D09193010C1727
:1015F0001D0720F0B8018BE10E947408B8016C1B34
:101600007D0B8AE10E94740820910E0130910F0138
:1016100040E050E06091060170910701809108015F
:10162000909109010E943D38109206011092070125
:101630001092080110920901B90187E00E94CF09B8
:1016400020910401309105019093050180930401DC
:10165000BC01621B730B8CE10E94740860910E0147
:1016600070910F018DE10E94740810920F01109289
:101670000E010E9434286093000170930101809351
:10168000020190930301DF91CF911F910F91089573
:1016900040E0A42FB0E0FD01EE0FFF1FEE0FFF1F93
:1016A000E851FE4FAA0FBB1FAC55BE4F2D913C9188
:1016B00080819181A281B381820F931FA11DB11DF1
:1016C00080839183A283B3834F5F413111F780916F
:1016D0002C0290912D02019690932D0280932C0262
:1016E0000E946A0A80912C0290912D028436910505
:1016F00011F40C942D0A08958F929F92AF92BF928D
:10170000CF92DF92EF92FF92CF93DF93CDB7DEB708
:1017100028970FB6F894DEBF0FBECDBFF82E5B0141
:1017200040E0682FCE0105960E948B0741E06F2DA7
:10173000CE0101960E948B0729813A8140E050E05A
:10174000CD80DE80E12CF12C2C193D094E095F097A
:10175000B50180E090E08F809884A12CB12C6819AD
:1017600079098A099B090E940D382B813C8140E050
:1017700050E0281939094A095B090E945F382C0D8D
:101780003D1D4E1D5F1D57FF03C020E030E0A90145
:10179000C90128960FB6F894DEBF0FBECDBFDF910A
:1017A000CF91FF90EF90DF90CF90BF90AF909F9040
:1017B0008F9008950C948609462FE82FF0E0EE0FE5
:1017C000FF1FE45AFE4F208131818250853130F471
:1017D000E82FF0E0E459FF4F608101C061E0C901EA
:1017E0000C944514825E0C9468078091550208950C
:1017F00080915302811112C00E947A07882381F0E0
:101800000E947D0720912F0230913002821B930BA2
:101810009C0181E02530310520F002C081E008956F
:1018200080E008950F931F93CF93DF9310E0CFEFE5
:10183000DFEF00E009C0812F0E94F20B8C179D079B
:1018400010F4EC01012F1F5F80915502181798F3D7
:10185000802FDF91CF911F910F910895CF93DF9348
:1018600090915302911104C0DF91CF910C94F20B2F
:1018700090913902C82FD0E0992391F00E94F20B89
:10188000CC0FDD1FFE01E65CFD4FCA5BDD4F208102
:10189000318148815981241B350B280F391F07C01E
:1018A000FE01EE0FFF1FE65CFD4F20813181C90173
:1018B000DF91CF910895CF93C82F80915302882351
:1018C00041F0C11106C00E947D07909330028093C1
:1018D0002F02C09353020E94342860933102709308
:1018E000320280933302909334020E9475098091F2
:1018F0005202811104C08C2FCF910C94D304CF914C
:10190000089580E00E945B0C81E08093520208956C
:101910000E94810C80E00C946605EF92FF920F9379
:101920001F93CF93DF9381E00E94660585E10E94BB
:1019300068078093550206E412E03AE3E32E32E0B2
:10194000F32EC0E0D0E00CC08C2F0E94F20BF80107
:10195000819391938F01F701819391937F01219658
:101960008091550290E0C817D90774F31092530282
:101970001092520280E00E945B0C10923002109292
:101980002F02109231021092320210923302109202
:101990003402DF91CF911F910F91FF90EF90089546
:1019A000FF920F931F93CF93DF93809154020E9475
:1019B0002E0CEC01F12C01E010E01CC08F2D0E94D8
:1019C0002E0CAC0180915302802321F0C417D5075F
:1019D00078F40DC020915403309155032F5F3F4F91
:1019E000369527952C0F3D1F2417350708F4102B2B
:1019F000000FF39480915502F81600F3812FDF91C8
:101A0000CF911F910F91FF9008951F93CF93DF9374
:101A1000EC0110E008C0812F825E0E9482078C17C3
:101A20009D0738F01F5F809155021817A0F381E0E1
:101A300001C080E0DF91CF911F910895BF92CF92B6
:101A4000DF92EF92FF920F931F93CF93DF938AE081
:101A500090E00E94050D882309F461C00E94120CD9
:101A6000809354020E94F20B8C0162E084E692E0C3
:101A70000E941C180817190750F17AE3E72E72E04C
:101A8000F72EE6E4CE2EE2E0DE2EC0E0D0E0BB246E
:101A9000B39416C08C2F0E94F20BF701819391939F
:101AA0007F01F601819391936F01801B910B20912F
:101AB0005403309155032817390708F4B12C2196A7
:101AC0008091550290E0C817D90724F302C0BB24C7
:101AD000B394109239020E943428609335027093B7
:101AE00036028093370290933802BB2059F0DF9181
:101AF000CF911F910F91FF90EF90DF90CF90BF900B
:101B00000C94810C0E94D00CDF91CF911F910F910A
:101B1000FF90EF90DF90CF90BF900C945B0CDF9123
:101B2000CF911F910F91FF90EF90DF90CF90BF90DA
:101B30000895CF9380913902811119C081E080937B
:101B40003902809154020E94F20BC0E00CC08C2F2D
:101B50000E94F20BEC2FF0E0EE0FFF1FEA5BFD4F4F
:101B600091838083CF5F80915502C81780F3CF9116
:101B700008950F931F930E9434280091350210910D
:101B800036022091370230913802601B710B820BB4
:101B9000930B28EE33E040E050E00E943D38C9014D
:101BA0001F910F91089583E090E00E94050D882316
:101BB000C9F080915302811103C00E941E0D12C012
:101BC0000E94990D0E94D00C90E0809590952091F4
:101BD000530230E082239323892B81F40E94B90DB4
:101BE0004F9760F40E94F80B882311F082E008956B
:101BF000809152028823D1F381E0089580E00E9411
:101C00005B0CF0CF1F93CF93DF93EC0110E00FC07C
:101C1000812F0E94F20B8C179D0710F081E00CC001
:101C2000812F0E942E0C8C179D07C0F71F5F80919B
:101C30005502181768F380E0DF91CF911F91089546
:101C40001F93CF93DF93EC0110E00FC0812F0E9410
:101C5000F20BC817D90710F081E00CC0812F0E9449
:101C60002E0CC817D907C0F71F5F809155021817AF
:101C700068F380E0DF91CF911F9108956091550244
:101C8000662321F070E00E94293802C060E070E015
:101C9000CB0108950E94C4100E94421E85E00E945C
:101CA000A5300E944F2988E00C94A5300E94C410F2
:101CB0000E94461E86E00E94A5300E944F2988E0BF
:101CC0000C94A530E0915602F091570285919491C1
:101CD000FC010994E0915602F091570232968591E9
:101CE0009491FC010994E0915602F09157023496C8
:101CF00085919491FC010994CF93DF931F92CDB706
:101D0000DEB7811107C00E941B1D0E946A0E0E944F
:101D1000560E0FC0813059F469830E941B1D0E942A
:101D20006A0E6981611105C00E944A0E02C081E0FD
:101D300001C080E00F90DF91CF910895BF92CF92C4
:101D4000DF92EF92FF920F931F93CF93DF938C015B
:101D5000C62E0E94620E0E94FD1C0E94A9290E94AC
:101D6000C410F12C82E0D82EC0E0D0E0EE24E39441
:101D70000E948A30811106C0F801EF0DF11D849197
:101D80000E94141F0E944E10B82E84E0B81209C0A1
:101D9000EF2DF0E03196E00FF11FE491E11123C047
:101DA00005C082E0B81202C0F110FA94EE2081F072
:101DB0000E94B329D82E6C2D0E947C0EE82E882319
:101DC00039F00E947D07C817D90779F4E11003C0E4
:101DD000C11016C0E12C81E0B812CACF0E941B1DB1
:101DE0000E946A0E0DC0F394E1CF0E947D07EC01C2
:101DF0000E94730ED82E6C2D0E947C0EE82EE6CF2A
:101E00008D2DDF91CF911F910F91FF90EF90DF907B
:101E1000CF90BF900895FC0124812052621710F4E6
:101E20000C946516862F90E0821B91090E94E2189F
:101E30006EE00C94021260E088E592E00E94631765
:101E400087FD0AC0811102C00C94C72D992787FD18
:101E5000909501970C943B2408950E94F4040E94ED
:101E600097310E942A2E62E471E082E391E00E94A1
:101E7000251E88EE93E00E94400780E00C94173600
:101E800060E571E088E592E00E94741685E890E0D4
:101E90009093590280935802ECE5F2E08081805ED5
:101EA00080830895CF93DF93EC010E94BC108B8157
:101EB0009C810E94FF110E94C0106A8188819981D3
:101EC000DF91CF910C949B11FC0187818F3118F425
:101ED0008F5F8783089586818F5F86830895FC01D5
:101EE0008781882319F081508783089586818150E6
:101EF000868308951F93CF93DF93FC01C681D0E0C2
:101F00006D2F80E00E94B6101C2F105F8C2FCF5FCA
:101F10000E9459128C2FC113FACFDF5FD23081F7A4
:101F2000DF91CF911F9108951F93CF93DF93EC0121
:101F300080EE90E00E943D151FEF8E81181721F072
:101F4000CE010E947A0F1E818F81682F70E094E08D
:101F5000759567959A95E1F78F700E94B6100E946B
:101F60004E10823049F0843019F0813049F413C0AA
:101F7000CE010E94640FE1CFCE010E946F0FDDCF32
:101F80008830D9F68D81E881F981E80FF11D8F81C4
:101F90009E81890F8083DF91CF911F910895FC016D
:101FA00071836083428334832383158280E2868336
:101FB00017820895CF93DF93EC0180EE90E00E94AA
:101FC0003D150E94C410CE010E94520F61E08D8128
:101FD0000E94B6100E944E108230B1F0843041F061
:101FE0008130C1F480EE90E00E94451580E026C06B
:101FF0004D81242F30E08A8190E00197281739071E
:102000002CF74F5F4D83E2CF8D818823F9F2815009
:102010008D83DCCF8830D1F682E00E94A51082301B
:1020200048F083E00E94A53080EE90E00E944515C4
:1020300081E004C0CE010E94940FC3CFDF91CF9105
:1020400008950C948206E0916202F0E0EE0FFF1F0B
:10205000E45AFE4F25913491C9010895CF93DF933F
:10206000D82F0E94820607C082E390E00E944007BA
:102070000E948206DC2FC82F8D13F6CF10926202C9
:102080001092610280936302882319F080E00E941D
:10209000B13080916302DF91CF910895EF92FF926A
:1020A0000F931F93CF93DF93C0E0D0E0F12C0AEFA2
:1020B00010E016C00E948206F82E81E090E00E9497
:1020C000400780916302F81202C0219609C08F2D4B
:1020D000DF91CF911F910F91FF90EF900C942E10F4
:1020E000E09062022E2D30E0220F331FF901E659F5
:1020F000FE4F65917491C8010E9429386F5F7F4F30
:10210000C617D707B8F2FF20B9F0409161024F5FC0
:1021100040936102F901E858FE4F85919491242F74
:1021200030E02817390740F085E08E1518F0E39469
:10213000E09262021092610280916302DF91CF917E
:102140001F910F91FF90EF900895CF93DF93D82FB9
:10215000C09163020E944E10909162029D1711F08F
:102160008C17C1F3892FDF91CF910895462F682FE7
:1021700080EE90E00C94541560E080E00C94B61072
:1021800061E080E00C94B61080EE90E00C94841531
:10219000CF93DF93FC01DB018C91882389F0C08110
:1021A000D1814883808191810196918380838C9134
:1021B00081508C93882321F00190F081E02D1082D2
:1021C000DF91CF910895BF92CF92DF92EF92FF926D
:1021D0000F931F93CF93DF93EC018B017A0141158D
:1021E000510501F1CA010E948A38F8019081B82E88
:1021F000981708F4B92ECB2CD12CA601B7018881F1
:1022000099810E949338288139812C0D3D1D398395
:102210002883F80180818B198083882319F0E88155
:10222000F9811082DF91CF911F910F91FF90EF9074
:10223000DF90CF90BF900895EF92FF921F93CF93BE
:10224000DF9300D000D0CDB7DEB77C01CA014B834D
:102250005C8369837A830E94D028182F69817A81F0
:10226000DB018C914B815C81811768F44FE3C701DE
:102270000F900F900F900F90DF91CF911F91FF90D3
:10228000EF900C94C810F70120813181210F311D8E
:1022900031832083DB018C91811B8C93882321F077
:1022A0000190F081E02D1082F9012AE030E00CC0AD
:1022B000CA01B9010E942938405DBAE06B9F4019FC
:1022C000112442931150AB011111F2CF0F900F90D6
:1022D0000F900F90DF91CF911F91FF90EF90089595
:1022E0000F931F93CF93DF93CDB7DEB72B970FB626
:1022F000F894DEBF0FBECDBF8E010F5F1F4F1A8750
:10230000098727E02B87AC01BE01655F7F4FCE01B7
:1023100009960E941C11B80180EE90E00E94AE3632
:102320002B960FB6F894DEBF0FBECDBFDF91CF91D5
:102330001F910F9108951F93CF93DF93CDB7DEB711
:1023400061970FB6F894DEBF0FBECDBF0097D1F0F6
:10235000162F613108F010E1412F50E0BC01CE0191
:1023600001960E94A238E1E0F0E0EC0FFD1FE10FC2
:10237000F11D1082BE016F5F7F4F80EE90E00E94E2
:10238000AE3601C080E061960FB6F894DEBF0FBE96
:10239000CDBFDF91CF911F9108951F93CF93DF930E
:1023A000CDB7DEB761970FB6F894DEBF0FBECDBFD5
:1023B0000097D1F0162F613108F010E1412F50E065
:1023C000BC01CE0101960E949338E1E0F0E0EC0FF1
:1023D000FD1FE10FF11D1082BE016F5F7F4F80EE88
:1023E00090E00E94AE3601C080E061960FB6F8948E
:1023F000DEBF0FBECDBFDF91CF911F91089560E189
:102400000C94CD11CF92DF92EF92FF920F931F9316
:10241000CF93DF93CDB7DEB762970FB6F894DEBFE8
:102420000FBECDBF009761F1613108F060E17C0122
:10243000CC24C394D12CCC0EDD1E86011CC0C70158
:102440006A8B0E94C138F80181938F01FFEFEF1A68
:10245000FF0A6A8981110FC0E1E0F0E0EC0FFD1F77
:10246000E60FF11D1082BE016F5F7F4F80EE90E09E
:102470000E94AE3606C0802F8C19861700F3ECCF71
:1024800080E062960FB6F894DEBF0FBECDBFDF913D
:10249000CF911F910F91FF90EF90DF90CF90089513
:1024A000882319F08AE891E002C08EE891E00C944C
:1024B000FF11682F80EE90E00C94B036CF93DF933D
:1024C0001F92CDB7DEB7682F06C080E269830E94F5
:1024D0005912698161506430C4F786E891E00F9029
:1024E000DF91CF910C94CD11CF93DF93D82FC0E023
:1024F00004C080E20E945912CF5FCD13FACF8C2F17
:10250000DF91CF91089580E10C9474126AE00E94EB
:102510001D38892F805D0C945912DF92EF92FF9243
:102520000F931F93CF93DF93EC01162F16160CF029
:1025300059C064E670E00E942938D62EE72ECB0100
:102540000E94D028082F23E0F22EF80E04C080E26B
:102550000E9459121150F116D4F3412F552747FD0F
:1025600050952F2D332727FD3095235031094217E1
:10257000530754F4812FDF91CF911F910F91FF905A
:10258000EF90DF900C945E128D2D9E2D0E947011A5
:10259000CE0164E670E00E942938EC01101B012F87
:1025A000015011161CF48EE20E945912102F115086
:1025B000101644F4CE016AE070E00E942938862F9C
:1025C0000E948612111674F4CE016AE070E00E9437
:1025D0002938DF91CF911F910F91FF90EF90DF90FD
:1025E0000C948612DF91CF911F910F91FF90EF9085
:1025F000DF900895CF92DF92EF92FF920F931F9397
:10260000CF93DF93EC01162FC42E16160CF088C062
:1026100068EE73E00E942938D62EE72ECB010E9487
:10262000D028F82E082F0C5F04C080E20E945912B7
:1026300011500117D4F31017DCF0C11019C0CE01EE
:102640000E94D028082F03C080E20E945912115026
:102650000117D4F3CE010E9470118DE6DF91CF9166
:102660001F910F91FF90EF90DF90CF900C94591233
:10267000412F552747FD5095202F332727FD3095B3
:1026800024503109421753075CF4812FDF91CF9119
:102690001F910F91FF90EF90DF90CF900C945E12FE
:1026A0008D2D9E2D0E947011CE0168EE73E00E9468
:1026B0002938EC011F19012F015011161CF48EE26C
:1026C0000E945912102F1150101644F4CE0164E6E6
:1026D00070E00E942938862F0E948612CE0164E69F
:1026E00070E00E942938EC01012F015011163CF4D2
:1026F0006AE070E00E942938862F0E948612101628
:102700007CF4CE016AE070E00E942938DF91CF911D
:102710001F910F91FF90EF90DF90CF900C94861255
:10272000DF91CF911F910F91FF90EF90DF90CF90AD
:1027300008956F927F928F929F92AF92BF92CF92A5
:10274000DF92EF92FF920F931F93CF93DF937C0161
:10275000962E742E822E16160CF044C021119A94D7
:10276000C7010E94D028C0E0D0E0082F10E0A92CBB
:10277000BB24A7FCB09404C0872D0E945912219657
:10278000692C6C1A6501CC1ADD0A0C151D05A4F321
:10279000882019F08DE20E945912C016D1068CF4DF
:1027A000862DDF91CF911F910F91FF90EF90DF90D9
:1027B000CF90BF90AF909F908F907F906F900C9430
:1027C0005E12C701DF91CF911F910F91FF90EF90A3
:1027D000DF90CF90BF90AF909F908F907F906F9041
:1027E0000C947011DF91CF911F910F91FF90EF909A
:1027F000DF90CF90BF90AF909F908F907F906F9021
:10280000089520E00C94991340E20C940114CF93A6
:10281000DF936CE370E00E9429389B01EC0140E3F8
:1028200063E0C9010E9401148AE30E94591240E347
:1028300062E0CE01DF91CF910C940114292F221F69
:102840002227221F19F091958195910940E20C945D
:102850009913161634F461500E948D1283E40C947F
:1028600059120895161634F461500E94041485E23A
:102870000C945912089563303CF062500E94041485
:1028800082E991E00C94FF110895CF93DF93C62F56
:1028900014167CF5642F6150C23071F028F4CC23FB
:1028A000B9F0C130C1F406C0C43059F080F0C53071
:1028B00091F409C0D6E510C0642FDF91CF910C943C
:1028C0002914D4EF06C00E941E1485E50EC0615085
:1028D000D1E440E002C0D5E541E00E94FA128D2F1C
:1028E0000E945912C33029F488E6DF91CF910C94ED
:1028F0005912DF91CF910895462F64E00C9445144E
:10290000462F61E00C944514462F60E00C9445146A
:10291000462F63E00C944514CF93DF93EC0160E005
:102920008E810E94B83781E090E00E94453761E0D7
:102930008E810E94B83781E090E00E94453760E0C8
:102940008E810E94B83784E690E0DF91CF910C949D
:102950004537CF92DF92EF92FF920F931F93CF9361
:10296000DF937C01C0E0D0E0C62ED12C87010C0F94
:102970001D1F61E0F80187810E948037B6010C2E8F
:1029800002C0759567950A94E2F761707727F801A0
:1029900087810E94B8372196C430D10539F7C70125
:1029A000DF91CF911F910F91FF90EF90DF90CF902B
:1029B0000C948C14CF92DF92EF92FF920F931F939F
:1029C000CF93DF937C01C0E0D0E0C62ED12C8701ED
:1029D0000C0F1D1F61E0F80187810E948037B6014E
:1029E0000C2E02C0759567950A94E2F761707727FF
:1029F000F80187810E94B8372196C830D10539F790
:102A0000C701DF91CF911F910F91FF90EF90DF9061
:102A1000CF900C948C141F93CF93DF93EC01162F5F
:102A2000642F8C810E94B8378D818F3F19F060E050
:102A30000E94B8378F85612F84FF06C0CE01DF91D9
:102A4000CF911F910C94DA1470E084E0759567952E
:102A50008A95E1F7CE010E94A914612FCE01DF9182
:102A6000CF911F910C94A91441E00E940B1581E0B5
:102A700090E0089540E00C940B15FC016089262F2E
:102A80002160208B69600C943A15FC0160896E7F8F
:102A9000608B68600C943A15FC016089262F2460D5
:102AA000208B6C600C943A15CF93DF93CDB7DEB7D3
:102AB00028970FB6F894DEBF0FBECDBF28E0E4E63E
:102AC000F0E0DE01119601900D922A95E1F7FC01EC
:102AD0002389421710F0422F4150E1E0F0E0EC0F63
:102AE000FD1F22E0429FE00DF11D11242081260FE1
:102AF0002068622F28960FB6F894DEBF0FBECDBFB8
:102B0000DF91CF910C943A1561E00E943A1580ED67
:102B100097E00C944537CF93DF93EC01423018F0E7
:102B20008F8588608F874B8B1C8A222329F0413048
:102B300019F48F8584608F8780E593EC0E94453778
:102B400060E08C810E94B83760E08E810E94B837C7
:102B50008D818F3F19F060E00E94B8376F8564FD6A
:102B60001DC063E0CE010E94A91484E991E10E9496
:102B7000453763E0CE010E94A91484E991E10E94E7
:102B8000453763E0CE010E94A91486E990E00E94D7
:102B9000453762E0CE010E94A91416C06062CE01E2
:102BA0000E943A1584E991E10E9445376F85606281
:102BB000CE010E943A1586E990E00E9445376F8564
:102BC0006062CE010E943A156F856062CE010E945C
:102BD0003A1584E0888BCE010E944C15CE010E94EC
:102BE000841582E0898B66E0CE01DF91CF910C9451
:102BF0003A156F927F928F92AF92CF92EF920F938E
:102C00001F93CF93DF93CDB7DEB73C01162F842FF0
:102C10005D854E853F859889F301848325830683EE
:102C2000E782C086A1868286538744873587968748
:102C300061E00E948037F30185818F3F19F061E0E8
:102C40000E94803761E0F30186810E948037112362
:102C500019F0F301178603C080E1F301878720E0B4
:102C600041E060E1C301DF91CF911F910F91EF909F
:102C7000CF90AF908F907F906F900C948B158F9228
:102C8000AF92CF92EF920F93DC0113961C921E929B
:102C90001297EBE8F0E0ED93FC931F921F921F92C6
:102CA0001F928C2CAE2CC02EE22E042F2FEF462F1D
:102CB00061E00E94F9150F900F900F900F900F9107
:102CC000EF90CF90AF908F900895DC011796ED9123
:102CD000FC911897B2E06B9FE00DF11D1124259136
:102CE0003491C9010C94FF110F931F93CF93DF937D
:102CF000EC018B01CB010E946728682FCE010E9456
:102D0000D71683E990E09983888318870F83DF9132
:102D1000CF911F910F910895DF92EF92FF920F9341
:102D20001F93CF93DF93EC01F62E69871A8681E01B
:102D30008D8382E0D82EEE24E3948E01075F1F4F2F
:102D40000E944E10482F823011F0843061F4E881E7
:102D5000F9810280F381E02D6F2DCE010995F9866E
:102D6000DA86ED8204C0813089F0883079F0C801BC
:102D70000E9463298111ED828D81882319F0CE0193
:102D80000E9405178A858F5F8A87DACF8FEF898740
:102D900081E08E838D83483009F080E0DF91CF9110
:102DA0001F910F91FF90EF90DF9008950895FC011F
:102DB00089E990E09183808312821382648381E0A9
:102DC000858386830895FC018281811103C081E09F
:102DD00082830895438190E0840F911D248130E027
:102DE000215031098217930714F44F5F43830895EC
:102DF000FC018281882319F08150828308958381A8
:102E0000882311F08150838308951F93CF93DF931C
:102E1000EC0110E0612F80E00E94B61080E20E9479
:102E20005912E881F9816B81610F0190F081E02DE9
:102E3000CE0109950E9483121F5F123059F76A81F3
:102E400080E00E94B6108EE30E9459126A818FE0E2
:102E50000E94B6108CE30E9459121D82DF91CF911F
:102E60001F9108950F931F93CF93DF93EC010E945E
:102E70004E10182F0E948A30882321F081E08D8324
:102E80001FE71BC00B818A81080F123031F014300C
:102E900039F4CE010E94E31603C0CE010E94F81659
:102EA0008B819A81890F081711F081E08D838D81C4
:102EB000882319F0CE010E940517812FDF91CF9151
:102EC0001F910F910895EF92FF921F93CF93DF937D
:102ED0001F92CDB7DEB77C0181E0F701858311E059
:102EE000C70169830E9432176981811102C0F7010D
:102EF0001682F7019681911108C0883031F481E083
:102F0000868383819281890F09C0662311F0F701BE
:102F10001583813029F79111E3CF8FEF0F90DF9167
:102F2000CF911F91FF90EF9008950F931F93CF9330
:102F3000DF93EC018B0150E00E941C114AE3B801C1
:102F4000CE01DF91CF911F910F910C94C810EF9299
:102F5000FF920F931F93CF93DF9300D01F92CDB7B3
:102F6000DEB78C01462F09969A8389838EE08B8386
:102F7000D801EC91F0E0EE0FFF1FEB56FE4FE5900D
:102F8000F490BE016D5F7F4FCE0101960E949517B0
:102F9000A701BE016D5F7F4FCE0101960E94E31035
:102FA00040E2BE016D5F7F4FCE0101960E94C810C6
:102FB000F80141815281BE016D5F7F4FCE010196C4
:102FC0000E941C114FE2BE016D5F7F4FCE01019642
:102FD0000E94C810D80117964D915C911897BE01B8
:102FE0006D5F7F4FCE0101960E941C110F900F90D4
:102FF0000F90DF91CF911F910F91FF90EF90089567
:1030000027E1289FB001299F700D112464577F4F3D
:1030100047E150E084E692E00C94B13827E1289F24
:10302000B001299F700D112464577F4F47E150E094
:1030300084E692E00C94CF38DC01EC91B5E0EB9F94
:10304000F0011124E60FF11DEE0FFF1FEB55FE4FAF
:1030500025913491C9010895CF93DF93EC010E942B
:103060001C184F815885849F9001859F300D949F37
:10307000300D1124C901DF91CF9108950F931F9353
:10308000FC01A181B28120914E0330914F030E9437
:10309000EF3724E630E040E050E00E943D388901FF
:1030A0009A01093EFDEF1F072105310520F008EECA
:1030B0001DEF20E030E0C8011F910F910895FC0141
:1030C0002081213029F420914A0330914B0309C01B
:1030D000223029F4209148033091490302C020E0B6
:1030E00030E0FC0187819085289FA001299F500D29
:1030F000389F500D1124CA010895E6E4F3E0808161
:1031000091810895FC016081F9E06F9FB001112465
:103110006B507E4F49E050E00C948138DC01EC911B
:10312000F0E0EE0FFF1FEB56FE4F25913491C901E1
:103130000C94CD1160E170E00C948E18CF93DF9366
:10314000EC01888160E0811108C0CE010E942C183A
:1031500067E00E94801487E011C0CE010E942C1805
:1031600065E00E9480148FE20E9459128F81988539
:103170000E94701183E40E94591288E0DF91CF9180
:10318000089566E0FC01838194810E94841486E0A6
:10319000089566E0FC01858196810E94841486E092
:1031A0000895FC0181819281883EFDEF9F0729F4FB
:1031B0008DE392E00E94FF1103C067E00E94881433
:1031C00088E0089547E1489F9001499F300D112400
:1031D0002B563F4FC90108950F931F93CF93DF9351
:1031E000CDB7DEB7A4970FB6F894DEBF0FBECDBF44
:1031F0008C01AB01BC01CE0101960E94971ACE0151
:1032000001960E94051B87E1FE013C96D8010190C2
:103210000D928A95E1F7A4960FB6F894DEBF0FBE23
:10322000CDBFDF91CF911F910F910895FC012081B7
:10323000260F283010F4208302C0FC0110820C9469
:1032400082180F931F9361E00E942C189C0140E0AC
:1032500050E060E074E887ED97E10E943D38890115
:103260009A0101328EE418072105310520F000E2B1
:103270001EE420E030E0C8011F910F9108950F93E4
:103280001F9361E00E942C189C0140E050E060E434
:1032900078E78DE791E00E943D3889019A0109386D
:1032A00083E118072105310520F008E813E120E04B
:1032B00030E0C8011F910F9108950F931F93CF9392
:1032C000DF9300D0CDB7DEB78C0169837A830E948B
:1032D0002119AC0169817A81C80103960F900F9082
:1032E000DF91CF911F910F910C9400290F931F93A1
:1032F000CF93DF9300D0CDB7DEB78C0169837A839B
:103300000E943F19AC0169817A81C80105960F902E
:103310000F90DF91CF911F910F910C94002961E0E4
:103320000E941C18BC0184ED92E60E942938CB0152
:1033300008950F931F93CF93DF9300D0CDB7DEB7DF
:103340008C0169837A830E948F19AC0169817A812B
:10335000C80107960F900F90DF91CF911F910F91A9
:103360000C940029CF93DF93EC010E948F192F81D9
:1033700038858217930710F498878F83CE010E94B7
:1033800021192B813C818217930710F49C838B8336
:10339000CE010E943F192D813E818217930710F4C0
:1033A0009E838D83DF91CF910895CF93DF93EC01BE
:1033B00048EE5DEF01960E94002989819A819C83E5
:1033C0008B832881233039F49C01369527953695D7
:1033D00027953C832B839E838D83CE01DF91CF91F4
:1033E0000C94B219DF92EF92FF920F931F93CF9339
:1033F000DF9300D01F92CDB7DEB749E050E06BE21B
:1034000072E084E692E00E94813884E692E00E94B5
:10341000B21900E010E05EE0D52E6DE6E62E62E027
:10342000F62EDB82FA82E982402F4F5FBE016D5F8C
:103430007F4FCE0101960E949517C8010E940E1879
:103440000F5F1F4F0032110561F70F900F900F9023
:10345000DF91CF911F910F91FF90EF90DF90089532
:10346000262F443019F06FEF7FEF02C061E070E06B
:10347000223089F028F4222341F02130A9F408C039
:10348000233061F0243081F40CC00B960C94161993
:103490000B960C9499190B960C94D5190B960C94C9
:1034A0005D190B960C94761908951F93CF93DF93B3
:1034B000EC01162F0E946516CE0109960E9458292C
:1034C000882311F0298501C02FEF332727FD309580
:1034D000812F90E02817390729F11230A9F028F43C
:1034E000112341F01130F1F40AC0133091F014307F
:1034F000C9F414C0CE010B960E949A1813C0CE01D5
:103500000B960E949E180EC0CE010B960E94D118F9
:1035100009C0CE010B960E94C11804C0CE010B96C3
:103520000E94C91880E0DF91CF911F910895EF921A
:10353000FF920F931F93CF93DF93EC018B017A01DE
:1035400061E772E00E9474168FEF89878FE990E03F
:103550009983888387E1F801DE011B9601900D9223
:103560008A95E1F7FBA2EAA2DF91CF911F910F911B
:10357000FF90EF9008950F931F93CF93DF93CDB7F4
:10358000DEB728970FB6F894DEBF0FBECDBF8C0113
:10359000BC016C5E7F4F21E832E04EE050E0CE018E
:1035A00001960E94CF0FCE0101960E94DA0F81E0B2
:1035B000F801858328960FB6F894DEBF0FBECDBF05
:1035C000DF91CF911F910F910895CF93DF93EC017D
:1035D0006AA17BA16F5F7F4F0B960E94A7170E9485
:1035E000C4100E94BC108CE892E00E94FF110E945F
:1035F000C0106EE0CE0144960E949B110E944F299C
:1036000083E0DF91CF910C94A530DF92EF92FF928F
:103610000F931F93CF93DF93CDB7DEB767970FB6A6
:10362000F894DEBF0FBECDBF8C0187E1D82E9BE0A2
:10363000E92EF12CE00EF11E60E0C8010E94631734
:1036400087FD2BC0853019F0863049F404C0C801CD
:103650000E94E51AF1CFC8010E94BB1AEDCFF70115
:10366000DE0111969D2D01900D929A95E1F7682F3C
:10367000C8010E948C16811109C0FE013196D70144
:103680008D2D01900D928A95E1F7D6CF83E00E94AF
:10369000A530C7010E94B219CFCF67960FB6F89434
:1036A000DEBF0FBECDBFDF91CF911F910F91FF9075
:1036B000EF90DF9008958091420390914303892B0E
:1036C000A1F08CE10E94680765E02AE0AC01249F2C
:1036D000C001259F900D11240E941E148DE60E94AA
:1036E000591283E40E94591204C08CE693E00E94B0
:1036F000FF110C9483128AE10E94680765E00E9422
:103700001E148DE60E94591286E50E9459120C94EF
:103710008312CF93DF9300D0CDB7DEB789839A832E
:103720000E94BC1089819A810E94FF110E94C010E2
:103730008091A1029091A2020E948A38892B51F0B7
:1037400085E593E00E94FF118091A1029091A20271
:103750000E94FF110F900F90DF91CF910C94831274
:1037600090E0880F991F62E088539D4F0C94CD1113
:103770000F931F93CF93DF9361E084E692E00E9462
:103780002C188C0162E084E692E00E942C18EC0177
:1037900083E10E9468078017910790F4C817D90742
:1037A00088F49C012C1B3D0BC8018C1B9D0B64E60F
:1037B00070E00E942938C9010E942938862F03C071
:1037C00084E601C080E0DF91CF911F910F910895B1
:1037D000613011F40C942E0C0C94DB25CF93DF9305
:1037E000D82FC62F825E0E940008882351F06C2FCC
:1037F0008D2F0E94E81B46E06C2FDF91CF910C9437
:10380000451485EE92E0DF91CF910C94FF110F9358
:103810001F93CF93DF93C82F162F0E94BC100E94D6
:10382000F80B811108C083E090E00E94050D882309
:1038300041F080E209C080913902882321F082E4BE
:1038400003C08DE601C082E60E94591280915302A6
:103850008823C9F0D0E001E080915402D81731F0FC
:1038600080915302802321F081E303C08FE501C0E2
:1038700080E30E945912000FDF5FD63069F780E2C3
:103880000E94591203C087E00E9474120C2F0F5F30
:10389000802F0E9486128AE30E945912612F8C2F7A
:1038A0000E94EE1B0E9483120E94C010DC2FDE5F7C
:1038B0008D2F0E9486128AE30E945912612F802F59
:1038C0000E94EE1B8C2F8D5F0E9486128AE30E945D
:1038D0005912612F8D2F0E94EE1BDF91CF911F9106
:1038E0000F910C94831288E10E94680768E00E949F
:1038F000881480E20C9459120E94BC1084E692E075
:103900000E943E1868E00E94881480E20E945912CA
:103910000E94C42567E00E9484140E9483120E94C2
:10392000C0108CEE92E00E94FF1167E080912803A6
:10393000909129030E9480140C9483120F931F937B
:10394000609186027091870280918802909189022D
:1039500020917B02222371F00E943428009186027C
:10396000109187022091880230918902601B710BAF
:10397000820B930B28EE33E040E050E00E943D388C
:10398000C9011F910F9108950E94FE21811110C05D
:103990000E945022882331F00E94FE2181110AC02A
:1039A00084E40BC00E94F80B811106C08EE405C0B0
:1039B00083E403C085E401C082E40E94591280E2DE
:1039C0000E9459120E949E1C0E94071480E20C94CF
:1039D00059120E94BC100E94731C67E086E10E948D
:1039E000DC0B0E9483120E94C0100E94C41C67E07E
:1039F00083E10E94DC0B0C9483120E9434286093B4
:103A000086027093870280938802909389021092B5
:103A10008202109283021092840210928502109208
:103A20007E0210927F02109280021092810281E049
:103A300080937B0208950F931F930E943428009176
:103A40008602109187022091880230918902601BC2
:103A5000710B820B930B60938602709387028093A5
:103A600088029093890210927B021F910F91089512
:103A70000E94042281111DC00E945622811119C08A
:103A80000E94F80B882351F1809182029091830269
:103A9000A0918402B091850280599F4FAF4FBF4FD4
:103AA0008093820290938302A0938402B093850254
:103AB000089580917E0290917F02A0918002B09142
:103AC000810280599F4FAF4FBF4F80937E029093EA
:103AD0007F02A0938002B0938102D2CF0895CF924B
:103AE000DF92EF92FF920E94BC1085EF92E00E945D
:103AF000FF110E949E1C0E9407140E94C01080E0CB
:103B000093E00E94FF116091820270918302809184
:103B100084029091850238EEC32E33E0D32EE12C3F
:103B2000F12CA70196010E943D38C9010E9407149B
:103B300083E093E00E94FF1160917E0270917F020A
:103B40008091800290918102A70196010E943D38E8
:103B5000C901FF90EF90DF90CF900C9407140E9462
:103B6000BC1086E093E00E94FF110E94E52568E00A
:103B70000E947C140E9483120E94C01082E10E9465
:103B80000008882349F08FE093E00E94FF110E9413
:103B9000EB2568E00E947C140C9483120E94BC10F8
:103BA00088E193E00E94FF1167E086E00E94DC0B51
:103BB0000E9483120E94C01080E293E00E94FF11D5
:103BC00047E061E080915003909151030E944514B9
:103BD0000C9483120E94BC1088E293E00E94FF11B3
:103BE00067E080E00E94DC0B0E9483120E94C010FC
:103BF0008FE293E00E94FF1167E082E10E94DC0BFC
:103C00000C9483120E94BC1086E393E00E94FF1183
:103C10008091420390914303892B29F065E087E06E
:103C20000E94DC0B04C08CE393E00E94FF110E9411
:103C300083120E94C0108EE393E00E94FF1165E0A2
:103C400085E00E94DC0B0C9483120F931F93CF939B
:103C5000DF9300D0CDB7DEB78B0189839A830E94B2
:103C6000C4100E94BC1089819A810E94FF110E9499
:103C7000C010C8010F900F90DF91CF911F910F914D
:103C80000C94FF1184E493E00C94891B8EE593E07F
:103C90000C94891B0E94BC100E94731C0E945B1B29
:103CA0000E94C0100E94C41C0C947B1B0E94BC107C
:103CB00085E793E00E94FF1167E08BE10E94DC0B37
:103CC0000E9483120E94C0108EE793E00E94FF11B1
:103CD0000C947B1B0E94BC1088E893E00E94FF11AB
:103CE0008091420390914303892B41F069E08091D8
:103CF0000401909105010E94291404C08EE893E00C
:103D00000E94FF110E9483120E94C01087E993E075
:103D10000E94FF110C945B1B6EEA73E081EA93E052
:103D20000C94251E0E948C1E0C944F296FEC73E09E
:103D30008EEB93E00E94251E88E893E10C944A28BC
:103D40000E94BC108AED93E00C94FF11CF930E9467
:103D5000BC1064E070E084E692E00E948E1880E27D
:103D60000E94591284E692E00E949E1880E20E940E
:103D700059128091A3020E94B01B0E94C0100E94A1
:103D8000B81B90E08436910569F48CE792E00E94BC
:103D90005829882321F084E00E9474120AC08BEE17
:103DA00093E005C062E00E94041480EF93E00E945B
:103DB000FF118CE792E00E945829882319F0C091E6
:103DC0007C0201C0CFEFC0FF05C065E080E00E942B
:103DD000DC0B03C085E00E94741280E20E9459123D
:103DE0008091640284508430A8F4C1FF05C065E06E
:103DF00082E10E94DC0B03C085E00E947412C2FFC6
:103E000005C00E942208CF910C94861280E2CF91C7
:103E10000C94591266E080916502909166020E94AE
:103E20008814CF910C94831290917D029F5F9093A0
:103E30007D02883049F168F48430E1F030F482305A
:103E4000A9F0B0F4813099F524C08630B9F0C0F4FF
:103E500013C08C3011F120F48A3039F1E0F417C02E
:103E60008E30F9F0E0F08F3011F51DC00C94E91C94
:103E70000C947C1C0C946F1D0C94021E61E005C018
:103E800061E083E00C94071C64E080E0FBCF64E019
:103E9000F8CF0C94A61E0C94AF1D0C94EA1D0C9444
:103EA000CE1D0C94561E0C946A1E0C944A1E089546
:103EB0008FEF80937C0208950F931F93CF93DF932E
:103EC0000E942822C0916702D091680261E084E6D6
:103ED00092E00E942C188C01CE0165E070E00E94F7
:103EE00029388FE00E947C0BEC0140E0BC01C80146
:103EF0000E940F268FE00E942326CE01DF91CF91F2
:103F00001F910F910C94122281E00C9436220E9492
:103F10006208882321F00E940D220C94CB2608957C
:103F200010928A020C945C1FCF93DF930E94871F2C
:103F30000E945D08EC0180918A02811111C062E04B
:103F400084E692E00E942C188C179D0748F481E0CB
:103F500080938A0280916702909168020E942222D7
:103F60000E9462088823D9F164E084E692E00E940E
:103F70002C188C179D0758F132C080918B02882332
:103F800089F08AE10E946807EC0184E692E00E94D1
:103F90005F18D195C195D1098C179D071CF481E05C
:103FA00094E017C080918C02811101C00EC08CE199
:103FB0000E946807EC0184E692E00E947D188C174D
:103FC0009D071CF485E094E004C082E00FC089EFF7
:103FD00093E09093A2028093A10281E007C08091B8
:103FE000100190911101029740F6EFCFDF91CF9130
:103FF000089580938C0260938B02089570939002D1
:1040000060938F0290938E0280938D0208950F9398
:104010001F93CF93DF93C0918D02D0918E02CE017A
:104020000E943E0E8C010E945D08C817D90738F423
:10403000C801DF91CF911F910F910C94200E81E068
:10404000DF91CF911F910F9108950F931F93CF93FD
:10405000DF930E940720182F0E945F22EC010E942C
:104060006208882311F001E001C0012F80919102C4
:10407000882329F0BE01812F0E947B2601C0812F59
:10408000882329F081E00E94B42281E00DC0011153
:1040900001C009C0BE01812F0E949A278C179D077D
:1040A00011F00E94982282E0DF91CF911F910F9131
:1040B00008950E94A6220E948D0C1092910280E128
:1040C0000C94232681E00E94B4220C94880CBC013D
:1040D00080E10E947C0B0C94B2250F931F93CF9329
:1040E000DF938C01EB010E94FE1FBE0180E10E9464
:1040F0007C0B40E0BC01C8010E940F26CE016AE0A3
:1041000070E00E942938CB01DF91CF911F910F9170
:104110000C9467200E948D0C0E9428228FE00C9442
:10412000232681E00E9436220C94880C0F931F9363
:10413000CF93DF931F92CDB7DEB78C018FE0498319
:104140000E947C0B4981BC01C8010F90DF91CF9187
:104150001F910F910C940F26BC018FE00E947C0BE5
:104160000C94B2250F931F93CF93DF93C091280334
:10417000D0912903CE010E943E0E8C010E945D0861
:104180008C179D0738F4C801DF91CF911F910F91D3
:104190000C94020E81E0DF91CF911F910F91089551
:1041A0001F93CF93DF930E94B220182F0E940D22FD
:1041B000EC01BC01812F0E947B26882329F081E03D
:1041C0000E94362281E01BC00E94620881110BC050
:1041D000111109C0CE010E94CC25811104C00EC06E
:1041E0000E9412220BC00E94F80B811107C0BE0171
:1041F000812F0E949A278C179D0791F782E0DF910B
:10420000CF911F9108950E9491200E9462200C94EA
:10421000880CCF93DF931F92CDB7DEB790919302B6
:10422000913039F018F0923081F406C00E94D0200D
:104230000CC00E94252009C00E94D30D823089F055
:1042400089830E94032189810CC0813051F49091AF
:104250009202992331F082E0809393020E948D0CA8
:1042600082E00F90DF91CF9108950E948D0C809194
:104270009402909195020E943E0E0E94200E882387
:1042800029F00E948A201092930208950E945920DA
:1042900081E080939102809393020895809392022B
:1042A00008950F931F93CF93DF93EC018A019093AE
:1042B00095028093940240E00E949620B801CE01BE
:1042C000DF91CF911F910F910C946D20FF920F936E
:1042D0001F93CF93DF9380E00E94000801E008273E
:1042E00080919602882381F00E94220890916B02AF
:1042F000FF24F394981301C0F12C11E0811110E018
:10430000913021F4112311F010E0F12C82E10E9490
:1043100000088823A9F082E10E946807EC0180E090
:104320000E946807C817D90728F49C012C1B3D0B75
:10433000E90102C0C81BD90BC53FD14008F001E01C
:10434000F11002C087E001C083E080937C0211235A
:1043500029F080917C02825080937C02002329F016
:1043600080917C02815080937C02F11004C0111175
:1043700002C0002311F081E001C088E00E94A53056
:104380000E942110811102C010929702F11008C002
:10439000111106C0011104C00E942110883041F0A3
:1043A00080919702823011F481E008C082E006C05B
:1043B000809197028F5F80939702F2CFDF91CF9128
:1043C0001F910F91FF9008950E94A62287E080938D
:1043D0007C0282E080937D020E949E3083E0809385
:1043E0009702089581E00E94B4228FEF80937C02AF
:1043F00088E00C94A53080939602089581E0909116
:104400009A02911180E0089581E020919802309104
:104410009902232B09F480E00895809198029091ED
:10442000990208959C01213088E0380710F020E0BF
:1044300038E03093990220939802C9010E94B70492
:104440000C948209BC018FE00E947C0B0C94122218
:1044500080919A02882349F080E090E00E94122225
:1044600081E00E94AD0410929A020895CF93C82F64
:1044700080919A0281110BC0CC2349F080E090E03A
:104480000E94122280E00E94AD04C0939A02CF9154
:10449000089580E090E00E94122281E00C94362280
:1044A00081E090919F02911180E0089581E0209138
:1044B0009D0230919E02232B09F480E008958091A3
:1044C0009D0290919E020895CF93DF93EC0140915D
:1044D000400350914103BA01645F714080EA92E069
:1044E0000E9473288091A002882311F0C0E0D0E0E0
:1044F000CE01DF91CF910895CF93C82F80919B0279
:1045000090919C020E94642220919D0230919E0213
:104510008217930711F4CC2349F090939E02809365
:104520009D020E94C504CF910C948209CF910895F9
:104530009C01213082E0380710F020E032E0309317
:104540009C0220939B0281E00C947C2280919F022C
:10455000882349F080E090E00E94982281E00E9448
:10456000B20410929F020895CF93C82F80919F02AA
:1045700081110BC0CC2349F080E090E00E9498228A
:1045800080E00E94B204C0939F02CF91089580E022
:1045900090E00E94982281E00C94B42280919F02C6
:1045A000811102C00C947C220895809164028730AE
:1045B00051F0982F9450943048F08150823048F454
:1045C00026EB32E008C024EA32E005C02DEA32E0F2
:1045D00002C02FEB32E0C90108958DE194E0909381
:1045E00057028093560290916402945081E0943077
:1045F00008F080E00E94FB2161E083E294E00E94E9
:104600009E0E91E0813009F090E0892F08950F937C
:104610001F93CF93DF930E944E2100916902109166
:104620006A02C0916702D091680263E084E692E07A
:104630000E942C18A801BE010E94512187E194E03C
:10464000909357028093560260E088E294E0DF91F5
:10465000CF911F910F910C949E0EEF92FF920F93AA
:104660001F93CF93DF938C01C7E6D2E0E880F980F7
:1046700061E084E692E00E942C1840E0B7010E94BD
:10468000962088819981B8010E942938CB010E9427
:10469000AC2081E194E0909357028093560260E051
:1046A00084E394E0DF91CF911F910F91FF90EF9001
:1046B0000C949E0ECF93DF93C0916702D091680255
:1046C00061E084E692E00E942C1841E0BE010E9465
:1046D000962081E194E0909357028093560260E027
:1046E00084E394E0DF91CF910C949E0E81E02091C1
:1046F000420330914303232B09F480E061E00E94E0
:10470000F91F83EF93E0909357028093560260E085
:1047100080E494E00C949E0E62E084E692E00E94B5
:104720002C186091690270916A02E0916B02F0911D
:104730006C024091520350915303E49F9001E59F16
:10474000300DF49F300D1124820F931F0E946D20B5
:104750008BE094E0909357028093560260E08BE4E4
:1047600094E00C949E0ECF93DF93C0916902D09198
:104770006A0262E084E692E00E942C18BE010E9468
:104780006D208BE094E0909357028093560260E096
:1047900087E594E0DF91CF910C949E0E8CE291E03E
:1047A000909357028093560260E080E694E00C9468
:1047B0009E0ECF93C82F8093A30225E634E030935A
:1047C000A2022093A1028D3030F4E82FF0E0ED55E5
:1047D000FF4F808101C080E0809361000E94003221
:1047E0000E94A5090E94ED22882309F43FC084E0BD
:1047F0000E94A530C53049F168F4C230D9F028F4E0
:10480000CC23A9F0C13081F52CC0C330B1F0C43045
:1048100059F516C0C83011F128F4C630C1F0C730C0
:1048200019F519C0CB3061F0CC30F1F406C08AE044
:1048300090E008C00E94CE2319C00E948C2316C0AD
:1048400085E090E00E942D2311C080E001C081E04E
:104850000E9407230BC00E94762308C00E94B32346
:1048600005C00E945A2302C00E94921E0E94B409F1
:10487000CF910C9410320F931F93CF93DF93EC01E1
:104880000E9400180E94D5228C0160E0C8010E949D
:10489000631787FD29C090916402E82FFF27E7FD89
:1048A000F095973019F4EA59FB4F0FC0892F8450C7
:1048B000843018F4E459FB4F08C09150923018F43A
:1048C000EC58FB4F02C0E758FB4F84918D3049F400
:1048D000BE0184E692E00E94EC18CE010E940E1800
:1048E000D1CF0E94D923D1CFDF91CF911F910F91CA
:1048F00008956CE774E08DEA92E00E9474166EE809
:1049000074E086EB92E00E9474166AE974E084EA2F
:1049100092E00E94741668EA74E08FEB92E00C94C7
:104920007416FC01428153814115510589F0A08123
:10493000B181B7FF03C0B195A195B10928EE33E06D
:104940000E94FB379A0140E050E00E943D3802C0CF
:1049500020E030E0C90108950F931F93CF93DF93B8
:1049600000D000D0CDB7DEB78C01862FF801628170
:1049700073810E94CF099C838B83F8018081918190
:104980009A838983CE0101960E9491240F900F9003
:104990000F900F90DF91CF911F910F9108950F937A
:1049A000FC01CA01002341F06417750708F4CB012C
:1049B0004617570748F409C04617570708F4CB01B4
:1049C0006417750708F401C0BA0197838683918341
:1049D0008083138212821582148233872287681B98
:1049E000790B718760870F910895FC019B0140E06E
:1049F00050E086819781281B390B41095109A28516
:104A0000B3850E94023820853185442737FD4095C3
:104A1000542F0E945F382115310581E04807510568
:104A20001CF457FD04C005C02FEF3FEF02C020E08B
:104A300030E0C9010895DF92EF92FF920F931F9328
:104A4000CF93DF93EC012A813B812417350720F4B3
:104A5000FA01E21BF30B03C0F901E41BF50B8C8197
:104A60009D81969587958E179F0788F588819981F6
:104A70008617970720F4FB01E81BF90B03C0FC0124
:104A8000E61BF70BEF2BF9F422C08A01021B130B74
:104A90007B01E81AF90A06C07C01E61AF70A8901C7
:104AA000041B150BC7010E94A128D82E8885998563
:104AB0000E94A128D8120BC01D830C83F986E886BA
:104AC0001B870A8704C024173507F8F2E5CFDF916A
:104AD000CF911F910F91FF90EF90DF900895CF92AB
:104AE000DF92EF92FF920F931F93CF93DF93EC012E
:104AF0008B019A01A885B9850E94FB372A853B85E1
:104B000040E050E00E945F386801E12CF12CC216B1
:104B1000D306E406F5061CF41F821E8204C0021BA5
:104B2000130B1F830E83DF91CF911F910F91FF9085
:104B3000EF90DF90CF900895EF92FF920F931F9325
:104B4000CF93DF93EC018B017A010E941B25A70113
:104B5000B801CE01DF91CF911F910F91FF90EF909F
:104B60000C946F2590932F0380932E0308958091CA
:104B7000CA02813029F420912E0330912F0302C004
:104B800020E030E0C901089560912A0370912B0361
:104B90008091CC020C94CF092091CF02213041F0BA
:104BA00041E020912E0330912F038217930708F0E4
:104BB00040E0842F08952CE0829FC0011124609171
:104BC000CC0288529D4F0C94AC246091CC0280E2C0
:104BD00093E00C94AC24CF93DF9300D000D0CDB7FA
:104BE000DEB780E00E9468079A83898382E10E9491
:104BF000680729813A81281B390B3A83298386E18A
:104C00000E9468079C838B83CE0101960E949124A9
:104C10000F900F900F900F90DF91CF910895909388
:104C200029038093280370932B0360932A03CB01FD
:104C30006AE070E00E94293870932F0360932E037E
:104C40004093CB020895EF92FF920F931F93CF935F
:104C5000DF9391E09093CA02FF24F3948F3009F020
:104C6000F12C8093CC0268EC70E00E947C0B909356
:104C70002D0380932C030E945D0820912E03309118
:104C80002F0340912803509129030F2DBC0188E187
:104C900093E00E94CF240E94F50B8093CD02809177
:104CA0002803909129030E943E0EEC0110E08CE055
:104CB000E82E12C0812F0E942E0CBC0120912E03E1
:104CC00030912F03E19EC00111240F2DAE018053BE
:104CD0009D4F0E94CF241F5F8091CD02181750F383
:104CE0001092CF021092CE02DF91CF911F910F91BF
:104CF000FF90EF9008950F931F93CF93DF93082FAA
:104D0000EB018091CB028823C9F040912C03509194
:104D10002D0320912E0330912F032417350708F41B
:104D20009A012C173D0710F4109252028091CF0285
:104D3000813021F00E94D30D8093CA028091CA0273
:104D4000813019F58091CF02823041F411E0209139
:104D50002E0330912F03C217D30708F010E00E94F2
:104D6000B7258C179D0778F0111103C0011101C000
:104D70000AC09091CE02892F8F5F8093CE0281E08E
:104D80009A3020F402C01092CE0280E0DF91CF91E1
:104D90001F910F9108950F931F93CF93DF93EC0111
:104DA0000E945D08AE01BC0188E193E00E949C2551
:104DB00010E00CE00DC0812F0E942E0CBC01019F61
:104DC000C0011124AE0180539D4F0E949C251F5F9E
:104DD0008091CD02181778F3DF91CF911F910F9139
:104DE0000895CF92DF92EF92FF920F931F93CF938C
:104DF000DF93609128037091290388E193E00E947A
:104E0000F524EC0180912803909129030E943E0E25
:104E10007C01D12C9CE0C92E12C0CD9C80011124B4
:104E200000531D4FB701C8010E94F524C817D907C8
:104E300028F0B701C8010E94F524EC01D3948091B9
:104E4000CD02D81650F3CE01DF91CF911F910F9173
:104E5000FF90EF90DF90CF9008950F931F93CF9323
:104E6000DF938B01809326039093270320912A03DD
:104E700030912B03EC012817390708F4E9010E944F
:104E8000B7259C018C179D0708F49E010217130794
:104E900019F18091CF028230A9F42017310790F0E8
:104EA00080912E0390912F0380179107A0F04091DD
:104EB00024035091250380912F02909130024817CE
:104EC000590749F080912F02909130029093250369
:104ED0008093240301C09801C901DF91CF911F91F4
:104EE0000F9108950F931F93CF93DF93EC010E94CE
:104EF0005D089093190380931803D0931B03C0930C
:104F00001A0310E00CE00DC0812F0E942E0C019FAF
:104F1000F0011124E053FD4F91838083D383C2833A
:104F20001F5F8091CD02181778F3DF91CF911F9109
:104F30000F9108951F93CF93DF93182FEB01CB01AF
:104F40000E94CB26CE010E9472270E94F1269093E8
:104F5000C9028093C802BE010E942D279C01809146
:104F6000CF02811110C0112389F08091CB028823D8
:104F700021F00E94810C1092520281E08093CF02B6
:104F800020E030E003C082E08093CF02C901DF91CE
:104F9000CF911F9108950F931F93009130031091AB
:104FA00031032091320330913303B801C9011F91BD
:104FB0000F91089512BE8DE78CBF88E083BF83B741
:104FC000836083BF89B7826089BF08958091300371
:104FD00090913103A0913203B09133030196A11D4A
:104FE000B11D8093300390933103A0933203B093AB
:104FF000330308950E94E6270E947E310E947229A1
:1050000080916200815019F080936200089581EED2
:10501000809362000E94CE220E9430080C94381DBA
:105020001F920F920FB60F9211242F933F934F931D
:105030005F936F937F938F939F93AF93BF93EF9300
:10504000FF930E94FA27FF91EF91BF91AF919F913B
:105050008F917F916F915F914F913F912F910F9021
:105060000FBE0F901F9018950F931F938FB7F89452
:1050700000913003109131032091320330913303BA
:105080008FBF3695279517950795B801C9011F91D0
:105090000F910895CF92DF92EF92FF92CF93DF931B
:1050A000EC010E9434286B017C01CC0EDD1EE11C5A
:1050B000F11C0E9434286C157D058E059F05C8F3F0
:1050C000DF91CF91FF90EF90DF90CF9008959C01FA
:1050D00080E001C08F5FF901459154912E5F3F4FF1
:1050E000452BC1F70895EF92FF920F931F93CF9333
:1050F000DF93EC017B018A0185E00E9468078E1531
:105100009F0518F4188281E007C00817190718F4E2
:1051100081E0888301C080E0DF91CF911F910F91E2
:10512000FF90EF90089521E030E09AE006C0A901D9
:10513000949F9001959F300D11248150C0F7C901B3
:10514000089597FD02C081E008958FEF0895CF92F2
:10515000DF92EF92FF92CF939B01AC016115710535
:105160008105910521F421E030E040E050E0C0E00D
:105170008AE0C82ED12CE12CF12CCF5FCA01B901F5
:10518000A70196010E943D382115310541055105C1
:10519000A1F78C2FCF91FF90EF90DF90CF900895E3
:1051A000BC0180E090E00C94A728FC0180819181F3
:1051B000860F971F97FF03C0118210820895242F36
:1051C00030E0281739071CF4408311820895918339
:1051D00080830895FC0180819181860F971F1816A6
:1051E00019061CF081E090E008C0242F30E0281759
:1051F00039071CF4408311820895918380830895B8
:10520000DF92EF92FF920F931F93CF93DF938C0166
:105210007A01DD24D394161617060CF0D12CF80170
:10522000C081D181BE0180E090E00E94A728823039
:1052300028F082500E9493289C0102C021E030E0B7
:10524000CE01B9010E942938009739F0DD2019F00C
:10525000281B390B04C09C010FC0DD2069F0C70179
:10526000821B930BC817D90718F47901EC0EFD1EA9
:10527000F801F182E0820BC02C173D0718F4C21B25
:10528000D30B02C0C0E0D0E0F801D183C083DF912E
:10529000CF911F910F91FF90EF90DF9008950E94A2
:1052A0004E108111FCCF0E944E108823E1F3089527
:1052B000FC01208127FD05C0818186958F5F81706B
:1052C000089580E00895FC01208127FD09C08181B7
:1052D000982F91509695282F269581E0921301C022
:1052E00080E0089585E00E94710720913403309199
:1052F00035032817390710F480E008C020913603E1
:10530000309137038217930718F481E00C94A004BE
:1053100008951F93CF93DF931FB7F894CEE3D3E0A4
:1053200068817981645F714085E00E947C0B909375
:105330003503809334036881798185E00E947C0B7A
:1053400090933703809336031FBFDF91CF911F9156
:1053500008956CE87EE680E00E947C0B9093390310
:10536000809338030895CF93DF9385E00E94680708
:1053700020914003309141032C503E4F28173907AC
:1053800018F48CE195E00CC080E00E947107209138
:105390003803309139032817390740F485E295E046
:1053A0009093A2028093A10280E041C086E00E9417
:1053B0006807EC0186E00E940008882359F180917B
:1053C000500390915103C817D90708F123C08C17D7
:1053D0009D0718F486E395E014C0809142039091F4
:1053E0004303892B11F482E022C087E00E94680702
:1053F000209144033091450328173907A0F78FE324
:1054000095E09093A2028093A10281E010C08EE209
:1054100095E0C6CF88E10E946807EC0184E692E03F
:105420000E943E18883E2DEF920789F6D6CFDF9175
:10543000CF9108950F931F93CF93DF938C01443046
:1054400019F0CFEFDFEF02C0C1E0D0E00E942310DF
:10545000D8011B96EC91F0E0EE0FFF1FE45AFE4FCF
:105460009C01C29FC001C39F900DD29F900D11243B
:1054700020813181820F931F91838083DF91CF91AF
:105480001F910F910895EF92FF920F931F93CF9367
:10549000DF931F92CDB7DEB78C01443021F0EE24AC
:1054A000EA94FE2C03C0EE24E394F12C69830E945D
:1054B0002310D8011B96ED91FC911C976981E60F92
:1054C000F11DE491F0E0EE0FFF1FE45AFE4F9C0146
:1054D000E29EC001E39E900DF29E900D112420816A
:1054E0003181280F391F318320830F90DF91CF91B5
:1054F0001F910F91FF90EF9008951F93CF93DF932B
:10550000EC01162F0E946516CE0109960E945829BB
:10551000882311F0898501C08FEF992787FD909529
:10552000612F70E08617970741F0EB85FC85E60F49
:10553000F71F84916D850E94DC0BDF91CF911F9145
:1055400008951F93CF93DF93EC01162F0E946516E9
:10555000CE0109960E945829882311F0298501C09F
:105560002FEF332727FD3095812F90E0281739073B
:1055700069F0111105C067E08B850E94DC0B06C045
:105580008B850E945F0767E00E940414DF91CF9132
:105590001F910895CF93DF9300D000D0CDB7DEB731
:1055A00080E00E945F079A83898382E10E946807F6
:1055B0009C838B83AE014F5F5F4F61E080E00E9470
:1055C000A9070F900F900F900F90DF91CF91089542
:1055D00060E070E088E495E00E94251E80E00E9473
:1055E0000008811106C00E944E108130B9F780E09A
:1055F000089581E00895CF93DF9300D000D0CDB718
:10560000DEB7862F5A8349833C832B83AE014F5FDD
:105610005F4F61E00E94A9070F900F900F900F90CD
:10562000DF91CF910895FF920F931F93CF93DF9354
:10563000F62E142F022F83E00E94A530812F0E94A6
:105640006807EC0181E080932E020E942907802FD9
:105650000E945F07AC019E01602F812F0E94FB2AF0
:105660000E942907FF2039F0DF91CF911F910F9100
:10567000FF900C94CA2ADF91CF911F910F91FF9058
:105680000895CF92DF92EF92FF920F931F93CF93E3
:10569000DF93CDB7DEB72E970FB6F894DEBF0FBEFF
:1056A000CDBF0E94A6220E94E82A882309F446C0A2
:1056B00069E575E08E010F5F1F4FC8010E947416E7
:1056C0008FEF8A8784EB90E09A8389838DE695E05B
:1056D0009D878C8789E08E87E02ED12E61E08E2D0C
:1056E0009D2D0E946317F82E87FD28C0082F1127D3
:1056F00007FD1095F801E359FA4FC49086E08F1525
:105700006CF38C2D0E940008882341F30E94290726
:1057100010922E026F2D8E2D9D2D0E948C168823A7
:1057200049F0F801EA58FA4F24914C2D61E08F2D91
:105730000E94132B81E080932E02D0CF81E00E9443
:10574000B4222E960FB6F894DEBF0FBECDBFDF9108
:10575000CF911F910F91FF90EF90DF90CF90089520
:105760000E94BC108DE795E00E94FF1165E08091DA
:105770003A0390913B030E9404140E9483120E94FA
:10578000C01085E895E00E94FF1167E086E10E9465
:10579000DC0B0C948312FF920F931F93CF93DF9334
:1057A000082F10923B0310923A03811105C00E940A
:1057B0002822C0E8D0E004C00E94A622C4E2D0E0C3
:1057C0000E94E82A811105C0C0E03AC0FF24F3948A
:1057D00001C0F12C0E94B02B0E944E10182F843073
:1057E00051F420913A0330913B032C173D0790F779
:1057F0002F5F3F4F0BC08230C1F420913A033091AC
:105800003B032115310531F32150310930933B031E
:1058100020933A0380913A0390913B03011103C016
:105820000E94122202C00E949822183019F4FF2010
:1058300089F205C0112351F2113031F2CBCFC1E012
:1058400081E0011103C00E94362202C00E94B422EE
:105850008C2FDF91CF911F910F91FF900895DF92D0
:10586000EF92FF920F931F93CF93DF9300D000D05E
:10587000CDB7DEB7162F7A01D22E0E94CB2B88230C
:10588000E9F083E00E94A530FC82EB828D2D0E941E
:105890005F079A838983AE014F5F5F4F612F8D2D24
:1058A0000E94A907802F0E945F079A838983AE0117
:1058B0004F5F5F4F612F802F0E94A9070F900F90BD
:1058C0000F900F90DF91CF911F910F91FF90EF906C
:1058D000DF900895FF920F931F93CF93DF93CDB77F
:1058E000DEB729970FB6F894DEBF0FBECDBF6DE8C7
:1058F00075E08E010F5F1F4FC8010E947416F02ED5
:1059000060E08F2D912F0E946317682F87FD0DC0D7
:10591000811103C042E350E002C048EE53E00FE0C3
:1059200022E080E00E942F2CEBCF29960FB6F8944E
:10593000DEBF0FBECDBFDF91CF911F910F91FF90C2
:105940000895FF920F931F93CF93DF93CDB7DEB7E8
:1059500029970FB6F894DEBF0FBECDBF63E975E09F
:105960008E010F5F1F4FC8010E947416F02E60E079
:105970008F2D912F0E946317682F87FD0DC0811115
:1059800003C042E350E002C04CE251E000E123E0FA
:1059900081E00E942F2CEBCF29960FB6F894DEBF42
:1059A0000FBECDBFDF91CF911F910F91FF90089552
:1059B0001F93CF93DF9300D000D01F92CDB7DEB7F7
:1059C000182F6D830E945F079A838983812F0E941D
:1059D00068079C838B83AE014F5F5F4F6D81812F82
:1059E0000E94A9070F900F900F900F900F90DF91DA
:1059F000CF911F910895EF92FF920F931F93CF9332
:105A0000DF93CDB7DEB72C970FB6F894DEBF0FBE8D
:105A1000CDBFF82EE62E69E975E08E010F5F1F4FAE
:105A2000C8010E9474168FEF8A872CEB30E03A830E
:105A30002983FC8661E0C8010E94631787FD12C0BC
:105A40008111F8CF10922E0260E0C8010E948C16DE
:105A5000882321F06E2D8F2D0E94D82C81E0809319
:105A60002E02E8CF2C960FB6F894DEBF0FBECDBF46
:105A7000DF91CF911F910F91FF90EF900895FF92CA
:105A80000F931F93CF93DF93CDB7DEB729970FB650
:105A9000F894DEBF0FBECDBFF82E6FE975E08E0122
:105AA0000F5F1F4FC8010E94741660E0C8010E947A
:105AB0006317682F87FD04C08F2D0E94FB2CF5CF44
:105AC00029960FB6F894DEBF0FBECDBFDF91CF9100
:105AD0001F910F91FF900895FF920F931F93CF9303
:105AE000DF93CDB7DEB729970FB6F894DEBF0FBEB0
:105AF000CDBF82E08093610065EA75E08E010F5FA3
:105B00001F4FC8010E947416F12E60E0802F9F2D58
:105B10000E946317182F87FD28C00E9400320E9440
:105B2000A509123091F02CF4112349F01130C1F481
:105B300009C0143079F064F0153091F40FC00E9460
:105B4000412B0EC00E946A2C0BC00E94A12C08C0E1
:105B500087E001C085E00E943F2D02C00E94D9333A
:105B60000E94B4090E941032D0CF83E0809361007C
:105B700029960FB6F894DEBF0FBECDBFDF91CF914F
:105B80001F910F91FF90089581E00C9417360F93A9
:105B90001F93CF93DF93CDB7DEB729970FB6F89455
:105BA000DEBF0FBECDBF6CE576E08E010F5F1F4FED
:105BB000C8010E94741660E0C8010E94631781301A
:105BC00049F0823051F081110BC08CE393E00E94C8
:105BD000482EF1CF0E946C2DEECF0E94C42DEBCF4A
:105BE00087FFE9CF29960FB6F894DEBF0FBECDBF71
:105BF000DF91CF911F910F9108950F931F93DC01B7
:105C00005C96ED91FC915D97EE0FFF1FEE0FFF1F6D
:105C1000EB57F94F0591159125913491B801C901C0
:105C20001F910F9108954EE150E069E976E00C94E0
:105C30008138FC01208931892630310520F025E0AA
:105C400030E0318B208B0895FC0180810E946D042F
:105C50000C9489294EE150E06EE673E08CE393E00A
:105C60000E94B1388CE393E00C94242E4EE150E076
:105C70006EE673E08CE393E00E94CF388CE393E010
:105C80000C94242E8CE393E00E94132E0C94362E59
:105C90000F931F93CF93DF93CDB7DEB7A9970FB6BE
:105CA000F894DEBF0FBECDBF8C01BC01CE010196C2
:105CB0000E94762ECE0101960E94932E8EE1FE0167
:105CC0003C96D80101900D928A95E1F70E94362EFC
:105CD000C8010E94242EA9960FB6F894DEBF0FBE0D
:105CE000CDBFDF91CF911F910F9108950F931F9317
:105CF000CF93DF93EC018B0167EB76E00E94741683
:105D00008FEF898784EC90E0998388838EE1F80196
:105D1000DE011B9601900D928A95E1F7DF91CF91FC
:105D20001F910F910895DF92EF92FF920F931F93AF
:105D3000CF93DF93CDB7DEB76E970FB6F894DEBF83
:105D40000FBECDBF7C018EE1D82E8701055F1F4FAE
:105D500060E0C7010E94631787FD2AC0803139F4D3
:105D6000C8010E94132E83E00E94A530F1CFF801F4
:105D7000DE0111969D2D01900D929A95E1F7682F05
:105D8000C7010E948C16811109C0FE013196D8010D
:105D90008D2D01900D928A95E1F706C083E00E9457
:105DA000A530C8010E94192EC8010E94242ED0CF10
:105DB0006E960FB6F894DEBF0FBECDBFDF91CF91C8
:105DC0001F910F91FF90EF90DF90089564E670E0CF
:105DD0000E942938CB0163E00E94041483E40C94F0
:105DE000591268EE73E00E942938CB0163E00E94EB
:105DF000041486E50C945912CF93DF9364E670E0A7
:105E00000E9429389B01EC0163E0C9010E9404143F
:105E10008EE20E945912CE016AE070E00E94293899
:105E2000862F0E94861289ED96E0DF91CF910C9427
:105E3000FF11CF93DF93EC012B9643E650E0CE01A8
:105E40000E940029CE01DF91CF910C94242EDC0119
:105E50009596ED91FC919697EE0FFF1FE352F94F47
:105E600025913491C9010C94FF110B960E94FD2DD0
:105E700024E630E040E050E00E943D3865E0C90192
:105E80000E94041480E30E94591280E30C9459127A
:105E90001F93CF93DF93EC01162F0E946516CE015E
:105EA00009960E945829882311F0298501C02FEFF7
:105EB000332727FD3095812F90E02817390709F403
:105EC0005FC01730B9F158F4133021F120F41130CC
:105ED000C9F0D8F413C0153021F140F51FC01B30B4
:105EE000F1F120F4193081F1A8F528C01D3009F432
:105EF00040C0C8F11E3009F043C03FC063E08B854D
:105F00009C851FC08D859E8502C08F8598890E94C3
:105F1000E62E36C089890E94501232C08B899C8936
:105F2000F6CF8D899E890E94FC2E2AC065E08F895C
:105F3000988D1CC065E0898D9A8D18C063E08B8DAB
:105F40009C8D0E9404141CC065E08D8D9E8D0E9466
:105F5000321416C08F8D98A10E94F12E11C066E0F8
:105F600089A19AA103C065E08BA19CA10E943B146A
:105F700007C0CE010E94272F03C0CE010E94352FFB
:105F8000DF91CF911F910895FC0124E6269FC00167
:105F9000279F900D112420813181820F931F843619
:105FA000910508F002C084E690E0918380838081AF
:105FB00091818D3A964220F08CEA96E2918380831B
:105FC0000895FC012AE0269FC001279F900D11240F
:105FD00020813181820F931F8A30910508F002C021
:105FE0008AE090E09183808380819181893E934013
:105FF00020F088EE93E0918380830895FC0128EEE1
:1060000033E0629FC001639F900D729F900D112439
:1060100020813181820F931F88352BE1920708F090
:1060200002C088E59BE191838083808191818133E7
:10603000954720F080E395E7918380830895FC01E4
:1060400080819181680F791F6330710518F0718329
:10605000608304C083E090E091838083808191819C
:10606000893C910520F088EC90E09183808308952D
:10607000262F443019F06FEF7FEF02C061E070E02F
:10608000273059F158F42330E9F020F42130A9F0F9
:10609000B0F411C02530D9F0E8F417C02B3051F11D
:1060A00020F4293001F118F51BC02D3059F138F1D9
:1060B0002E3079F52AC00C94192F0D9601C00F9639
:1060C0000C94C42F41E0419622C04396F9CF4596E7
:1060D0000C94E12F44E147961AC044E1499617C059
:1060E00045E04B9602C04AEF4D960C94EA284F9635
:1060F0000C94FE2F48EE53E081960C940029839671
:106100000C941F3044E0859602C044E087960C94BE
:10611000D5280895CF930E94B909C82F882349F044
:1061200080915A03811102C00E94A01E87E00E9444
:10613000A530C0935A038C2FCF9108950E94CB278E
:1061400070935F0360935E03089590915B039817CB
:1061500021F080935B030C949E30089588E00C94AA
:10616000A53090915B03983011F40C94A5300895FC
:106170009B01220F331F281739075CF06817790736
:106180001CF4281B390B07C01816190614F49C01BF
:1061900002C020E030E0C9010895969587958531C9
:1061A000910520F46AE070E00C94B8300E94AE30A3
:1061B00080E090E008950F931F93CF93DF93EC015D
:1061C000D695C795D695C795C93CD1052CF00E94A8
:1061D000AE3020E030E00FC06AE070E0CE010E94F7
:1061E000B8308C016AE070E0CE0188970E94B83028
:1061F0009C01200F311FC901DF91CF911F910F9199
:10620000089560ED77E00E9429386AE070E00C9410
:10621000B8306AE070E00E942938CB016D38710512
:1062200020F464E170E00C94B8300E94AE3080E05D
:1062300090E008956AE070E00E9429389B01CB014C
:1062400068E270E00E942938283B314020F464E184
:1062500070E00C94B8300E94AE3080E090E0089579
:106260006AE070E00E9429389B01CB0168E270E08F
:106270000E9429382135310520F464E170E00C9446
:10628000B8300E94AE3080E090E008956AE070E09F
:106290000E9429389B01CB0168E270E00E942938F6
:1062A000283B314020F464E170E00C94B8300E9447
:1062B000AE3080E090E0089520915B032330A9F098
:1062C00020F4213061F068F408C0253061F068F0F6
:1062D000263079F0273079F40AC00C94CD300C9434
:1062E00001310C9409310C941A310C94DB300C946C
:1062F00030310C94463180E090E008950E94CB2725
:1063000020915E0330915F03CB01821B930B0E94AF
:106310005C3120915C0330915D038217930731F06B
:1063200090935D0380935C030C94A4040895CF9331
:10633000DF931F92CDB7DEB7E0919804F0919904F6
:10634000309729F4ECE9F4E002C0219303C0CE01B8
:1063500001962EEB8E179F07C0F70F90DF91CF911C
:106360000895CF93DF9300D0CDB7DEB78091980426
:1063700090919904009711F48CE994E09E012F5FAD
:106380003F4F281B390BC9010F900F90DF91CF9120
:106390000895CF93DF931F92CDB7DEB72091980475
:1063A000309199042115310511F42CE934E0F901FB
:1063B000CE010196AF01421B530B8E179F0728F0A9
:1063C00060816E3B11F43196F5CFCA010F90DF91D9
:1063D000CF9108958CE393E00E94FD2DAB01BC01A9
:1063E00089E693E00C94EA3489E693E00E94313424
:1063F00089E693E00E945F3560E08AE00C94803784
:1064000080916300813059F4809156039091570335
:10641000892B29F00E94EA3182E08093630008957D
:1064200080916300813029F00E94F43181E08093F3
:1064300063000895CF93C82F682F89E693E00E94E8
:10644000B036909160039C2790936003CF9108959C
:106450008BE30C941A32CF93DF93EC0102C00E94BD
:106460001A3289918111FBCFDF91CF9108950F935B
:106470001F93CF93DF93CDB7DEB72B970FB6F8946A
:10648000DEBF0FBECDBF8E010F5F1F4F1A8709877A
:1064900027E02B87AC01BE01655F7F4FCE010996D7
:1064A0000E941C11C8010E942B322B960FB6F89443
:1064B000DEBF0FBECDBFDF91CF911F910F91089529
:1064C000CF93DF93EC011092600384E20E941A32B2
:1064D000CE010E9437320E9428328091610090E004
:1064E0000E9437320E9428326091610370916203EA
:1064F000809163039091640328EE33E040E050E024
:106500000E943D38C9010E9437328EE20E941A3241
:1065100060916103709162038091630390916403C1
:1065200024E630E040E050E00E943D38CA01B90165
:106530002AE030E040E050E00E943D38CB010E946C
:106540003732DF91CF910C9428328DE00E941A32BD
:106550008AE00C941A328091600390E00E943732F6
:106560000C94A532CF93DF9381E090E00E946032DB
:10657000C0E0D0E0FE01E255F84F84910E94680728
:106580000E9437320E9428322196CE30D10591F7F1
:10659000C0E08C2F0E94DB250E9437320E942832F7
:1065A000CF5FC630B1F70E94E5250E9437320E94C6
:1065B00028320E94EB250E9437320E942832DF9158
:1065C000CF910C94AB32CF93DF93D82F82E090E041
:1065D0000E946032C0E08C2FDD2319F00E945F071B
:1065E00002C00E9468070E9437320E942832CF5FA3
:1065F000C43289F78091530290E00E9437320E94A2
:1066000028328091C8029091C9020E9437320E94BC
:106610002832DF91CF910C94AB3283E090E00E945E
:1066200060320E94C9310E9437320E9428320E9493
:10663000B1310E9437320E9428320C94AB32CF9392
:10664000DF93C0915603D09157030E94B232C230FB
:10665000D1056CF081E0C430D1050CF480E00E94DB
:10666000E332229721F0DF91CF910C940D33DF912B
:10667000CF9108950F931F9380916300813051F162
:106680000E94342820916300223051F46093650306
:10669000709366038093670390936803109263007E
:1066A00000916503109166032091670330916803A0
:1066B000DC01CB01801B910BA20BB30B8093610318
:1066C00090936203A0936303B09364031F910F91AF
:1066D0000C941F331F910F9108950F931F93CF9325
:1066E000DF931F92CDB7DEB78A0169830E941A3209
:1066F0006981862F90E00E9437328DE30E941A3222
:10670000C8010E9437320F90DF91CF911F910F91F6
:106710000C94A5321F93CF93DF9300D000D0CDB758
:10672000DEB788EC90E00E942B320E94A53247E051
:1067300050E060E085E40E946D3341E050E061E0AC
:1067400085E40E946D3342E050E062E085E40E94FF
:106750006D3310E040E0612FCE0101960E948B075F
:1067600049815A81612F81E60E946D334B815C81A2
:10677000612F82E70E946D3341E0612FCE010196C7
:106780000E948B0749815A81612F81E40E946D33F9
:106790004B815C81612F82E50E946D331F5F113157
:1067A000C9F60F900F900F900F90DF91CF911F912E
:1067B00008950E94EA310E948A330E94A5320E9405
:1067C0008A330E94A5320C94F431FC0184859585AE
:1067D000FC01F39520813181FC01EE5FFE4F808149
:1067E0009181281B390B3327C9010895FC01848549
:1067F0009585FC01F39540815181FC01EE5FFE4FD0
:10680000208131814217530741F00190F081E02D42
:10681000E80FF91F208130E002C02FEF3FEFC901E0
:106820000895FC0184859585FC01F3954081518193
:10683000FC01EE5FFE4F208131814217530769F062
:10684000A081B181A80FB91F2C91808191810196FF
:1068500099279183808330E002C02FEF3FEFC90179
:106860000895FC0181A1882329F0A489B5898C9120
:1068700086FFFBCF11A20895CF93DF93FC012685FD
:106880003785D901B3958D919C91119701969927E0
:10689000E901CE5FDE4F4881598184179507D9F30E
:1068A0000D90BC91A02DA20FB31F6C93A685B78548
:1068B000B39511969C938E93A689B7892C9181E00C
:1068C00090E0078C02C0880F991F0A94E2F7282BEA
:1068D0002C9381E081A30488F589E02D8081806478
:1068E000808381E090E0DF91CF91089508951F9219
:1068F0000F920FB60F9211242F933F934F938F93C4
:106900009F93EF93FF935A991AC04CB180918B04D7
:1069100090918C040196992720918D0430918E04DA
:106920008217930769F0E0918B04F0918C04E5578E
:10693000FC4F408390938C0480938B0401C08CB1F6
:10694000FF91EF919F918F914F913F912F910F90D8
:106950000FBE0F901F90189589E693E00E94E533D3
:10696000892B11F00C94763408951F920F920FB674
:106970000F9211242F933F938F939F93EF93FF9345
:1069800020918B0430918C0480918D0490918E0421
:106990002817390711F4559812C0E0918D04F09131
:1069A0008E04E557FC4F208180918D0490918E04D8
:1069B0000196992790938E0480938D042CB9FF91B2
:1069C000EF919F918F913F912F910F900FBE0F905C
:1069D0001F901895CF92DF92EF92FF92CF93DF93A3
:1069E000EC016A017B01411581EE580761057105D3
:1069F000F9F0EC89FD8981E090E008A002C0880FE1
:106A0000991F0A94E2F7808360E079E08DE390E0DB
:106A1000A70196010E943D382150310941095109D1
:106A20005695479537952795211580E1380798F0B9
:106A3000EC89FD89108260E874E88EE190E0A7019E
:106A400096010E943D38215031094109510956955E
:106A5000479537952795E889F9893083EA89FB8935
:106A6000208319A2EE89FF89408181E090E09C019A
:106A70000D8C02C0220F331F0A94E2F7422B408391
:106A8000EE89FF8940819C010E8C02C0220F331FCA
:106A90000A94E2F7422B4083EE89FF8920810F8C14
:106AA00002C0880F991F0A94E2F7809582238083A1
:106AB000DF91CF91FF90EF90DF90CF900895CF932B
:106AC000DF93FC0186859785DC01B395EC01CE5FF1
:106AD000DE4F4D915C911197288139814217530700
:106AE000C1F7A689B7894C9181E090E09C01058CA3
:106AF00002C0220F331F0A94E2F7209524232C931F
:106B0000A689B7894C919C01068C02C0220F331FC5
:106B10000A94E2F7209524232C93A689B7892C9117
:106B2000078C02C0880F991F0A94E2F78095822390
:106B30008C9384859585FC01EE5FFE4F2081318129
:106B4000FC01F39531832083DF91CF91089510925A
:106B50006C0310926B0388EE93E0A0E0B0E08093AA
:106B60006D0390936E03A0936F03B093700383ED56
:106B700090E090936A03809369038BE893E090938D
:106B8000760380937503909378038093770380E472
:106B900090E090937A038093790329E230E0309378
:106BA0007C0320937B032BE230E030937E03209321
:106BB0007D032AE230E03093800320937F0390939B
:106BC0008203809381038CE290E09093840380930E
:106BD000830384E08093850383E08093860387E0CA
:106BE0008093870385E08093880381E08093890305
:106BF00008950F931F93CF93DF9300D0CDB7DEB7E7
:106C00008C0169837A830E94C93869817A818617E9
:106C1000970729F0C8010E94F03881E001C080E0A8
:106C20000F900F90DF91CF911F910F910895CF9307
:106C3000DF93C82F6DEC77E08CEB97E00E94251E68
:106C400067E070E080E090E00E94F93581111DC09E
:106C5000C1111BC061E070E08AE890E00E94F93544
:106C600081111BC0C11119C0D0E062E070E08CE658
:106C700093E00E94F935811118C0D11116C0CC23C0
:106C8000F9F0DF91CF910C94961E87ED97E00E946A
:106C9000FF110E94C007C1E0DDCF8AED97E00E949E
:106CA000FF110E94F219D1E0E0CF8DED97E00E9434
:106CB000FF110E94422E80ED97E00E944A28DFCF0C
:106CC000DF91CF9108950E944F370E942D0FCCEA9B
:106CD000D4E30E941B0F2097E1F30E94AC34F9CF5C
:106CE000CF92DF92EF92FF920F931F93CF93DF9398
:106CF0006C01EB017A01E60EF71E00E010E00BC01C
:106D00006991D601ED91FC910190F081E02DC601D1
:106D10000995080F191FCE15DF0591F7C801DF91FE
:106D2000CF911F910F91FF90EF90DF90CF9008953A
:106D30006115710581F0DB010D900020E9F7AD01CF
:106D400041505109461B570BDC01ED91FC9102802B
:106D5000F381E02D099480E090E008950C9498363A
:106D6000DC01ED91FC910190F081E02D09941F93DD
:106D7000CF93DF93182FEB0161E00E9480372097BB
:106D800011F460E004C0CF3FD10539F461E0812FF8
:106D9000DF91CF911F910C94B837E12FF0E0E052D2
:106DA000F84FE491E33071F018F4E130E1F405C0FC
:106DB000E43071F0E530B9F411C083B7806183BF6E
:106DC000CCBF15C08FB580688FBDDBBDCABD0FC0FD
:106DD0008FB580628FBDD9BDC8BD09C085B5806241
:106DE00085BDC3BD04C0C038D10584F6CACFDF91CC
:106DF000CF911F9108951F920F920FB60F921124F9
:106E00002F933F938F939F93AF93BF9380918F0462
:106E100090919004A0919104B091920430919704C4
:106E2000232F2D5F2D3720F40196A11DB11D05C024
:106E3000232F2A570296A11DB11D209397048093FA
:106E40008F0490939004A0939104B0939204809146
:106E5000930490919404A0919504B09196040196A6
:106E6000A11DB11D8093930490939404A093950465
:106E7000B0939604BF91AF919F918F913F912F91C5
:106E80000F900FBE0F901F901895019739F0880F43
:106E9000991F880F991F02970197F1F70895789429
:106EA00083B7826083BF83B7816083BF89B7816006
:106EB00089BF1EBC8EB582608EBD8EB581608EBDD1
:106EC0008FB581608FBD85B5846085BD85B58064D3
:106ED00085BD329A319A309A379A1AB8089584301B
:106EE00039F0853049F0833051F48FB58F7702C087
:106EF0008FB58F7D8FBD089585B58F7D85BD089534
:106F0000CF93DF9390E0FC01E35FF74F4491FC01E6
:106F1000E65CF74F8491882341F190E0880F991F38
:106F2000FC01EF58F74F25913491D9018959974FBA
:106F3000FC0185919491C82FD92F9FB7F8948C911B
:106F4000611106C0409584238C938881842308C0F6
:106F5000623041F4242F209582238C938881842BE6
:106F6000888302C0842B8C939FBFDF91CF910895BB
:106F70000F931F93CF93DF931F92CDB7DEB7282FC8
:106F800030E0F901E052F84F8491F901E35FF74FE7
:106F90001491F901E65CF74F04910023D1F08823A6
:106FA00021F069830E946F376981E02FF0E0EE0FD6
:106FB000FF1FE959F74F85919491DC019FB7F89431
:106FC0008C91611103C01095812301C0812B8C939A
:106FD0009FBF0F90DF91CF911F910F910895A29FB6
:106FE000B001B39FC001A39F01D0B29F700D811D5E
:106FF0001124911D08950E94EF37B7FF0895821B59
:10700000930B08950E94EF37A59F900DB49F900DAC
:10701000A49F800D911D11240895DB018F939F93F0
:107020000E940238BF91AF91A29F800D911DA39F36
:10703000900DB29F900D11240895991B79E004C022
:10704000991F961708F0961B881F7A95C9F78095A7
:107050000895AA1BBB1B51E107C0AA1FBB1FA6179F
:10706000B70710F0A61BB70B881F991F5A95A9F7F1
:1070700080959095BC01CD010895A1E21A2EAA1B1E
:10708000BB1BFD010DC0AA1FBB1FEE1FFF1FA217D8
:10709000B307E407F50720F0A21BB30BE40BF50BD5
:1070A000661F771F881F991F1A9469F7609570955E
:1070B000809590959B01AC01BD01CF010895052EEF
:1070C00097FB16F4009407D057FD0DD00E943D3871
:1070D00007FC09D07EF490958095709561957F4F5F
:1070E0008F4F9F4F089550954095309521953F4F74
:1070F0004F4F5F4F0895EE0FFF1F0590F491E02D65
:107100000994FB01DC0102C005900D9241505040F2
:10711000D8F70895FC0105900020E9F78095909537
:107120008E0F9F1F0895FB01DC014150504048F035
:1071300005900D920020C9F701C01D9241505040AA
:10714000E0F70895FB01DC014150504048F0019008
:107150000D920020C9F701C01D9241505040E0F748
:107160000895DC01CB01FC01E199FECF06C0FFBB15
:10717000EEBBE09A31960DB20D9241505040B8F7F7
:107180000895E199FECF9FBB8EBBE09A99278DB3FE
:107190000895A8E1B0E042E050E00C94B338DC017F
:1071A000A40FB51F4150504048F0CB01840F951FEC
:1071B0002E910E94E03841505040D0F70895262F7C
:1071C000E199FECF9FBB8EBBE09A01970DB20216EC
:1071D00031F02DBB0FB6F894E29AE19A0FBE0895F4
:1071E0000196272F0E94E0380C94DF38F894FFCFE7
:1071F000FF03E10100004000140054000000010200
:10720000010201010101010101000005010101016B
:1072100000000000000B0F00000000341570360065
:10722000000000651600000000D6160000000055A2
:107230001A301A05060807050909050700000507A1
:10724000000000007D2A432A00000000A12A1A2A1B
:1072500000000000482F3830563D302E33320000F9
:107260000000003C347036E5331134F6333134001D
:00000001FF
